:100000000C9466000C9487000C9487000C94870075
:100010000C9487000C9487000C9487000C94870044
:100020000C9487000C9487000C9487000C94870034
:100030000C9487000C9487000C9487000C94870024
:100040000C9487000C9487000C9487000C94870014
:100050000C9487000C9433030C9487000C94870055
:100060000C9487000C9485120C9487000C948700E4
:100070000C9487000C9487000C9487000C948700E4
:100080000C9487000C9487000C9487000C948700D4
:100090000C94691A0C9487000C9487000C948700C8
:1000A0000C9487000C9487000C9487000C948700B4
:1000B0000C9487000C9487000C9487000C948700A4
:1000C0000C9487000C9487000C94870011241FBEA9
:1000D000CFEFD1E2DEBFCDBF00E00CBF14E0A0E067
:1000E000B2E0EAE1F1E900E00BBF02C007900D9237
:1000F000AC33B107D9F717E0ACE3B4E001C01D920F
:10010000AB32B107E1F70E945B0C0C948B480C9466
:100110000000109242048091420480934104809137
:100120004104809340048091400480933F041092E6
:1001300043040895EEE6F0E080818260808383E0EE
:1001400084BD85BD8AEF87BD089508950895809187
:100150007100817008959B01AC01CA01AA27BB27D9
:10016000BC01892B79F0687F672B59F483E05695A1
:100170004795379527958A95D1F73093A00420931A
:100180009F0408953093A00420939F0408958091C4
:100190009E04982F9295969596959370282F221FDE
:1001A0002227221F9227282F22952F709227282F4F
:1001B0002695269592279170880F892B80939E040F
:1001C00008959093900480938F0485EB9BE3909324
:1001D000A6048093A50483E393E19093AC048093F9
:1001E000AB0485E694ED9093A2048093A104089556
:1001F00080918F0490919004AC01440F452F441FCF
:10020000550B5195482759276091A5047091A60474
:100210007093900460938F048091AB049091AC0430
:100220009093A6048093A5042091A1043091A20488
:100230003093AC042093AB04C901002496958795B4
:100240000794969587950794982F802D822793275A
:1002500084279527542F44275295550F507E842785
:1002600095279093A2048093A104660F771F6F5F78
:100270007F4F869F9001879F300D969F300D1124F0
:10028000C9010895FC019081992351F08091C80023
:1002900085FFFCCF9093CE00319690819923B1F7E2
:1002A00008951F93CF93DF93182F492FE0E1F7E2D2
:1002B000C0E0D0E0812F942FBF010E9442489B01F3
:1002C0006115710589F5812F942FBF010E94424865
:1002D000182F492FCF016AE070E00E944248FB01CD
:1002E0002196C430D10531F73097A1F18091C80033
:1002F00085FFFCCF812F942FBF010E944248605D93
:100300006093CE00CF016AE070E00E9442489B01FA
:1003100061157105F9F0812F942FBF010E944248A9
:10032000182F492FF901E2CF8091C80085FFFCCF3B
:10033000822F805D8093CE00812F942FBF010E9479
:100340004248182F492FCF016AE070E00E944248CE
:10035000FB01CACFDF91CF911F910895982F9F7015
:100360009A3040F48091C80085FFFCCF905D909357
:10037000CE0008958091C80085FFFCCF995C9093D2
:10038000CE000895CF93DF93EC01892F99278295B2
:100390008F700097C1F48D2F9927009789F4CE01B3
:1003A000929582958F7089279F708927009711F009
:1003B0000E94AE018C2F0E94AE01DF91CF91089573
:1003C0000E94AE01ECCF0E94AE01E5CF982F809144
:1003D000C80085FFFCCF9093CE0080E090E00895A8
:1003E0002091C800332727FD30952227330F221F85
:1003F0003327C90108958091C80087FFFCCF809101
:10040000CE0090E008959C018FEF8093940493E0D8
:10041000283E390768F5809391048093920424362E
:100420003105D8F0C90164E670E00E94424860934B
:100430009104C9016AE070E00E944248CB016AE081
:1004400070E00E94424880939204C9016AE070E023
:100450000E9442488093930408952A30310548F75A
:10046000C9016AE070E00E944248809393040895B5
:100470001092910410929204109293040895909116
:1004800044049360909344048093450408958091BC
:1004900044048360809344040895F999FECF92BD8B
:1004A00081BDF89A30B5F999FECF019692BD81BD14
:1004B000F89A20B5932F80E030E0282B392BC90122
:1004C0000895F999FECF92BD81BDF89A80B508953F
:1004D000F999FECF92BD81BD60BDF894FA9AF99A60
:1004E00078940895FF920F931F938C01F62E672F37
:1004F0000E946802C80101966F2D0E9468021F9138
:100500000F91FF9008958091C90088618093C90080
:1005100083E38093CC001092CD008091C80087FDCA
:1005200032C08091C90080688093C9008091C10069
:1005300088698093C1008FE18093C4001092C50048
:1005400090EC91B98CE382B987E384B995B99FEFB8
:1005500097B988EF8AB98BE08BB982E08DB99EB9E3
:1005600010BA91BB13BA94BB8DB581608DBD81E586
:100570008CBD08958091CE008AE00E94E90E8091A2
:10058000C80087FFCECF8091C80087FDF3CF809150
:10059000C80087FFF8CFEECFEF92FF920F931F9323
:1005A000CF93DF93EC0181E0CD32D80708F440C04F
:1005B000CCE2D1E07E0100E010E080918B049091CC
:1005C0008C048C179D0719F0CE010E94241AD09339
:1005D0008C04C0938B04D0939D04C0939C046091C1
:1005E000090270910A0280910B0290910C02A801FD
:1005F00097010E9469486FEF7FEF8FEF9FEF0E9496
:100600006948CA01B90128EE33E040E050E00E9499
:100610001748609398047093990480939A04909378
:100620009B04DF91CF911F910F91FF90EF90089560
:10063000C431D10508F0BECFC4E1D0E054E1E52ECD
:10064000F12C012D112DB9CF85E090E00E944D02D3
:100650000E94CC0280918B0490918C049093A4040E
:100660008093A30408951F920F920FB60F920BB6BA
:100670000F9211242F933F934F935F936F937F9328
:100680008F939F93AF93BF93EF93FF9340B14270CB
:1006900090B18091A904481749F1892F81704423B2
:1006A00009F4CAC0882309F4CAC09FEF8091F803F7
:1006B0008823D1F080914B04882309F4F0C0913055
:1006C00009F00DC180919C0490919D040796909330
:1006D0009D0480939C048D52914030F08CE291E017
:1006E00090939D0480939C044093A90480915B04A3
:1006F0008F3F29F080915B048F5F80935B04809132
:100700005C048F3F29F080915C048F5F80935C04D0
:1007100080918604909187048F5F9F4F49F080916C
:1007200086049091870401969093870480938604B1
:1007300080916A0490916B048F5F9F4F49F0809184
:100740006A0490916B04019690936B0480936A0401
:1007500080913C04823009F485C0813009F471C075
:10076000882309F056C08091010290910202A09165
:100770000302B09104028093050290930602A093B5
:100780000702B093080220910102309102024091C9
:100790000302509104028091980490919904A091D1
:1007A0009A04B0919B04820F931FA41FB51F8093DE
:1007B000010290930202A0930302B09304022091DD
:1007C0000102309102024091030250910402809193
:1007D000050290910602A0910702B0910802281725
:1007E00039074A075B07A8F480914D048F5F809317
:1007F0004D0480914D04817080934D0480914C0490
:100800008F5F80934C0480919C0490919D040E9482
:10081000CC02FF91EF91BF91AF919F918F917F910A
:100820006F915F914F913F912F910F900BBE0F9061
:100830000FBE0F901F901895882309F436CF91E0D2
:1008400035CF99B19295917080915904981709F319
:1008500090934D049093590480914C048F5F809342
:100860004C04D7CF8091550490915604892B89F27E
:10087000809155049091560401979093560480936B
:1008800055048091550490915604892B11F61092CD
:100890004D0480914C048F5F80934C04BACF292F74
:1008A000332727FD309580919C0490919D04280F5B
:1008B000391F30939D0420939C0481E02D3238072A
:1008C00008F00CCF2431310508F00ECF84E190E020
:1008D00090939D0480939C044093A90407CF9F3F6D
:1008E00009F002CF80919C0490919D04079790930A
:1008F0009D0480939C04449708F0F6CEE7CFCF92F6
:10090000DF92EF92FF920F931F93CF93DF93F894B0
:1009100080913C04813009F49BC480918204813031
:1009200009F49DC280913F048C3060F010923F0426
:10093000809140048F5F80934004809141048F5FD9
:100940008093410480914104882341F080914104C7
:1009500090E083709070892B09F410C2809142045A
:10096000883038F01092420480913C04882309F4C6
:10097000E4C1809141048F708093410490914004C0
:10098000809100029817C0F01092400480914304B7
:100990008F5F80934304909143048091AA04981739
:1009A00008F0FCC1809144048260809344048091EB
:1009B000480481608093480480912507882329F4A6
:1009C00080914004882309F4DFC18091400488238A
:1009D00029F480918204823009F46CC28091E80489
:1009E0008C3009F42BC280913C04882309F0D0C0DC
:1009F000909154048091F503981710F010925404CC
:100A00008091540480FFBEC05C9880918304209143
:100A1000F5034091F50390E030E0240F311D82177B
:100A2000930714F010928304809183046091F5037E
:100A300066950E943648992309F4BAC0DD24809156
:100A4000E804873009F4C0C0883008F469C18B30ED
:100A500009F4BAC08C3008F43BC28C3009F46BC383
:100A60008D3009F4B1C080918204823009F4E1C371
:100A700080912507882321F082E0D81609F4E4C389
:100A800080912507882309F40CC280916F048F7030
:100A900080936F048091410490E08370907002977E
:100AA0000CF4FBC185E20E943D1680916F0490E03A
:100AB0008370907002970CF4EDC18FEF8093670400
:100AC00080917804882309F07EC180918104882375
:100AD00071F080914504882351F08091A704813002
:100AE00009F429C28091A704882309F414C28091D3
:100AF0004604882309F055C180914B04882349F0AE
:100B000080913C04882329F48091F803882309F01C
:100B1000DCC20E941418DD2031F080913D048F5F0B
:100B2000817080933D04809183048F5F8093830460
:100B3000809119078F5F8093190780913F048F5F21
:100B400080933F04809154048F5F809354042091DC
:100B500019078091F50330E086958695869548E1E2
:100B6000849FC00111242817390714F01092190727
:100B70007894DF91CF911F910F91FF90EF90DF90CC
:100B8000CF9008955C9A88EF0E94F40F80913C0406
:100B9000813009F448C1823009F037CF80914D048B
:100BA000882309F431CF5C9A88EF0E94F40F2DCF8F
:100BB00080913D04882309F4BDC0DD24D394809145
:100BC000E804873009F040CF81E0D81609F4C3C1AA
:100BD000E2E0DE1609F047CF80916F048F5F8093CB
:100BE0006F0480912507882309F494C08091AC0597
:100BF000882309F5109219078091B005882349F4DC
:100C000080911B07882329F080917804882309F0BC
:100C10000CC68091340660917C06680F8091C006F6
:100C20009091C1060E94ED2910926F048091730487
:100C3000882309F427C58091AC05E091C006F091A6
:100C4000C106E80FF11D808180938A04809197048A
:100C50008093950480918A04807480939704809196
:100C60007804882309F0AFC480918A048F708F3094
:100C700009F4FEC480918A048F708F3029F180912D
:100C80008A040E94112A0091C606080F10918A0456
:100C9000107860919504802F412F0E947E1D1123B2
:100CA00009F0EEC480E0902F935F982B8091490467
:100CB000981751F08091490480934A049093490415
:100CC000809149040E94A80F8091E804833009F4C0
:100CD0006DC48091E8048730E9F480914604813046
:100CE00009F49BC58091940590919505E091A50527
:100CF000F0E0EE0FFF1FE35FFD4F60817181829591
:100D00009295907F9827807F98270E944248862F4F
:100D10000E94ED1680914404816080934404A3CE28
:100D2000813008F4A0CE843008F44ECF853009F02D
:100D30009ACE4ACF52E0D52E82CE20918B043091AC
:100D40008C048091A3049091A4042817390709F416
:100D500010CE80912507882309F00BCE85E20E94F2
:100D6000051660918B0470918C047093A4046093B9
:100D7000A30485E090E00E947202FBCD80914204C2
:100D80008F5F80934204EACD80918204823009F023
:100D90001CCE109282040E94523217CE109243044D
:100DA00001CE0E94BB198091410480FDA5CEE09147
:100DB0004104E695F0E0E370F070EF56FB4F808160
:100DC0000E94B01999CE8CE20E94112A982F80912E
:100DD0006F048111945F80911907882341F48091F9
:100DE0007904882309F4A1C383E20E940516809147
:100DF0001907843009F069CE80917904882379F449
:100E000080917604823008F4ABC3809138060E944A
:100E1000112A40913806407860E00E947E1D83E2EE
:100E20000E943D1652CE80914D04882309F4EDCDE9
:100E300088EF0E94F40F80913C04ADCE809148046D
:100E400080FF0AC080912507882309F027C280917E
:100E50005004882309F014C310924804C4CD809133
:100E60002507882311F50E94523280913C04882383
:100E7000F1F41092420480914204809341048091E5
:100E80004104809340048091400480933F04109279
:100E900043040DC01092670413CE85E20E9405162C
:100EA00004CE81E20E943D16F0CD0E940C2E1092DD
:100EB000820438CD8091E804853009F48FCD1092FA
:100EC000830410923D041092AC051092820486CDEA
:100ED000883009F0C8CDF1E0DF1609F42CC382E0B8
:100EE000D81609F0C0CD8091890480933E0480918A
:100EF0008804809389040E94C700809388048091AD
:100F000089048F7360E040E00E947E1D8091890417
:100F10000E94A80FA8CD8091440480FFE8CD809165
:100F200044048E7F809344040E94C9168091AC05CE
:100F30000E94D716DCCD8091440481FFD3CD8091EF
:100F400044048D7F809344040E94C9168091430419
:100F50000E94D716C7CD8091B0058F5F8093B005F2
:100F600080912507882309F47ECD8091AC058F5FA1
:100F70008093AC059091AC058091F703981710F021
:100F80001092AC058091AC05882309F06EC0809169
:100F9000E804833009F4AEC210E08091E8048730A1
:100FA00009F42AC381E00E94BC2980917C068F5FEE
:100FB00080937C06C0907C0690917C0680913A06D6
:100FC000981708F443C080917304882319F481E0D2
:100FD000809380048091E804813009F46EC380918D
:100FE000E804823009F465C382E00E94BC291092B3
:100FF000B00580917804882369F08091760480930D
:101000001B0780911B07882329F01092760481E04A
:101010008093AA0510927C068091E804833009F43D
:101020009FC38091E804873009F45EC380913B063A
:10103000882309F045C3909118078091AB05981754
:1010400029F080917304823008F423C480917C06D7
:1010500090E082959295907F9827807F982782587C
:10106000994F9093C1068093C0068091780488239D
:1010700009F0F9CC8091AC05E091C006F091C10671
:10108000E80FF11D808180938A0480918A048F701B
:101090008F3009F4AEC2809197040E94951D809113
:1010A0004A04882309F09EC280919704882309F09E
:1010B000DACC80914904882309F4D5CC8091490485
:1010C0000E94CE0F10924904CECC0E94C9166091A6
:1010D0008B0470918C04603A710508F4A0C1603AE9
:1010E000710509F452C280E090E02EE030E040E06B
:1010F00050E00E941748685E7E4F8F4F9F4F28E157
:1011000031E040E050E00E946948022F293008F4A5
:101110007FC318E0812F0E94D7161F5F1017D0F3EE
:10112000003108F0F6CC102F812F0E94E2161F5FCD
:101130001031D0F3EECC0E94C9168091480480FD96
:101140006AC180915004882309F05FC1E1E0DE1696
:1011500009F4EEC0F2E0DF1609F085CC80916F044F
:101160008F5F80936F0480912507882309F47BCCDF
:10117000E0917C06F0E0EE53F94F808184FDFBC1E5
:1011800086E08093F5038091AC05E091C006F09174
:10119000C106E80FF11D808180938A048091970435
:1011A0008093950480918A04807480939704809141
:1011B0008A048F708F3009F4F1C180918A048F7096
:1011C0008F3071F080918A040E94112A9091C60696
:1011D0006091950440918A044078890F0E947E1D99
:1011E00080914704982F92959F709093D706982FDF
:1011F0009770909334068695869586958170809336
:10120000180780911807882309F0AEC188E00E9472
:10121000051681E00E943D160E94BD17809134069C
:101220008F5F0E945D17809125078170809325074D
:101230001ACC81E20E943D1680913F0463E00E9437
:101240003648992309F021CC81E20E9405161DCC75
:101250000E9415138823A9F080918104882309F046
:1012600074C11092420480914204809341048091A1
:101270004104809340048091400480933F04109285
:1012800043040E942713882309F447CB80918104EB
:10129000882309F442CB0E940C2E3FCB8091250776
:1012A000823008F4D9CD80915004882329F48091AC
:1012B0009805882309F4D0CD809151048093470488
:1012C00090917C069F5F90937C0690917C06917034
:1012D00090937C0660917C0670E062957295707FB9
:1012E0007627607F76276258794F7093C1066093A6
:1012F000C00690917C06C92FD0E00E94572CCE5397
:10130000D94F8883E0917C06F0E0EE53F94F80815D
:101310008F708F5F8093F703E0917C06F0E0EE53CF
:10132000F94F808184FD0FC18CE08093F50394CD4B
:1013300080912507882309F496CB8091AC058F5FB7
:101340008093AC0580915004882309F401C19091E9
:101350005104809147048917D1F1F0907C06F394F1
:10136000FE220F2D10E0E801C295D295D07FDC2738
:10137000C07FDC27C258D94F80915104BE010E9422
:10138000572C0E53194FF8018083E0917C06F0E052
:10139000EE53F94F2081F801808190E030E0822700
:1013A000932784FD14C08091510480934704F092E8
:1013B0007C06E0917C06F0E0EE53F94F80818F705F
:1013C0008F5F8093F703D093C106C093C0068091CE
:1013D000AC056091F7030E9436489093AC0580916C
:1013E000AC05E091C006F091C106E80FF11D8081C7
:1013F00080938A0480918A048F708F3009F4BDC075
:10140000809197040E94951D2ECB809150048150AD
:101410000E94D7169BCE8FE00E94D71692CE80E016
:1014200090E02EE030E040E050E00E9417486E501F
:1014300070408040904028E131E040E050E00E9460
:101440006948022F222309F430C110E0812F0E9445
:10145000E2161F5F1017D0F3083008F028C1102FD4
:10146000812F0E94D7161F5F1830D0F3103108F07B
:1014700050CB812F0E94E2161F5F1031D0F349CB71
:1014800080915104809347040E94523280913C0421
:10149000882381F410924204809142048093410495
:1014A00080914104809340048091400480933F04E4
:1014B0001092430480917C068F5F80937C0680911C
:1014C0007C06817080937C0660917C0670E062955A
:1014D0007295707F7627607F76276258794F709378
:1014E000C1066093C00680917C06C82FD0E0809131
:1014F000470403CF809194059091950501969093B0
:1015000095058093940520919405309195058091DF
:101510009F059091A0052817390708F43DCD10923A
:1015200095051092940511E038CD892F60E040E0D8
:101530000E947E1D59CC80E00E94951D80918904F7
:101540000E94CE0F90CA80E1F0CE0E94523289CE26
:1015500080919805882309F03ACF0E940C2E37CF4E
:1015600080E00E94951D5BCC88E00E943D1681E0E2
:101570000E94051651CE88E004CE809197048823FE
:1015800009F08FC0109297043BCF0E94C91687E0E4
:101590000E94D71688E00E94D716BBCA80918A04A1
:1015A0008F7080938A041092970407CE809146042E
:1015B000813009F08ECB809194059091950501962C
:1015C0000E94030286CB8091340660913A064091D6
:1015D000AD0520913B060091B105E090AB050E945E
:1015E000031972CB80914A040E94CE0F10924A04D4
:1015F0005BCD109297044FCD80916E04813009F03D
:10160000D1CC609118078091340640917C062091DE
:10161000C606480F8CE995E00E94FF1E8091A50543
:10162000609194057091950540919C050E94651FFD
:1016300080919405909195050196909395058093DE
:101640009405E091A5052091940530919505F0E071
:10165000EE0FFF1FE35FFD4F80819181281739074F
:1016600008F4A0CC10926E0483E20E943D169ACC3E
:1016700080918A048F7080938A0410929704FACA2A
:1016800080E811CB8091340660913A064091AD0517
:1016900020913B060091B105E090AB050E94031933
:1016A000CACA81E00E94951D6DCF10E0D9CE102FDF
:1016B000DDCE81E08093800497CC809380048FCC32
:1016C0000E94A92980917304823008F0BFCC8091D8
:1016D000D706609118074091340620913A060EE72C
:1016E00016E00E94B42CB2CC80916E04813009F0D7
:1016F0009DCC809198058823B9F010926E041092C9
:1017000098058091A50560919405709195050E94BA
:101710003C1F8091A5050E94C81F9093A00580934F
:101720009F0583E20E943D1680919905882309F464
:101730007DCC109299058091A505609194057091DA
:1017400095056C190E942C1F8091A5050E94BF1F52
:101750009093A7058093A60580E00E943D1666CC75
:1017600080919805882309F07BC080919905882392
:1017700009F450C010929505109294058091E304ED
:101780008093A5058091A5050E94C81F9093A00590
:1017900080939F058091A5050E94BF1F9093A70588
:1017A0008093A6052091A6053091A70580919F05FD
:1017B0009091A0052817390720F01092A7051092E4
:1017C000A60580919905882309F055C08091A5054B
:1017D00060919405709195050E94192080939C0555
:1017E0008091A50560919C0543EF55E02BEA35E01B
:1017F0000DEA15E09FEBE92E96E0F92E0E94DF1E20
:1018000081E080933B068091BF068093C60609CC99
:1018100018E08ACC1123A9F2ADCF80919405909164
:10182000950501960E9403025DCA81E00E94951D04
:1018300080E00E94951D60913A068EE796E048EDA3
:1018400056E022EB35E00E941C2B109278048AE0CF
:101850000E942D2A1092970482E00E94E90ED9C9B5
:1018600010929805109295051092940583E20E94BB
:101870003D1611E07ACF109299058091A6059091BE
:10188000A705909395058093940580E00E943D16EE
:101890009DCF8091AB058093180719CF07C0809129
:1018A0004C04815080934C040E947F0480914C042E
:1018B0008823A9F70895AF92BF92CF92DF92EF925B
:1018C000FF920F931F93DF93CF93CDB7DEB760974F
:1018D0000FB6F894DEBF0FBECDBF0E9483020E94F8
:1018E000240380916E00826080936E0083E084BD4B
:1018F00085BD8AEF87BD8EE796E09093C106809301
:10190000C006F999FECF82E090E092BD81BDF89AC1
:1019100080B5982F937090933C048295817080934A
:101920007904F999FECF87E090E092BD81BDF89AE5
:1019300080B5882311F0813208F080E180930002A5
:10194000F999FECF83E090E092BD81BDF89A80B511
:101950008F708093C004F999FECF84E090E092BD2F
:1019600081BDF89A80B58F708093AD0488E090E0D7
:101970000E944D0280939E0420918B0430918C0430
:10198000280F391F3093900420938F0485EB9BE33D
:101990009093A6048093A50483E393E19093AC0411
:1019A0008093AB0485E694ED9093A2048093A10408
:1019B0000E94F8000E94F8000E94F800BC0188E034
:1019C00090E00E947202F999FECF8AE090E092BD09
:1019D00081BDF89A90B5892F8F708093A70480916C
:1019E000A704833010F01092A70492959F709F5F18
:1019F0009093AA048091AA04823018F482E0809324
:101A0000AA04F999FECF8DE090E092BD81BDF89ACD
:101A100060B5862F8C59893C08F410C160ED72E1E5
:101A200083E190E0F8946093090270930A02809336
:101A30000B0290930C020E94AE2D789400E010E00F
:101A40001DC08091ED040E94D7160E941418C80191
:101A5000849668E270E00E9456480E94AA190E948B
:101A60003D1680E10E94E90EC80187709070892BB5
:101A700069F00F5F1F4F0C32110579F0083208F73B
:101A8000802F0E94AA190E940516DBCF0E945315D1
:101A90000F5F1F4F0C32110589F70E94B4160E9488
:101AA00014180E94531580E00E948E13882331F091
:101AB00083E00E948E13882309F019C183E00E94FD
:101AC0008E13882309F0CAC08091ED048093D70655
:101AD000109218071092AB051092340681E08093A3
:101AE0003A0610923B068091D70660911807409104
:101AF000340620913A060EE716E00E94B42C60915D
:101B00003406C8010E94ED290E9478290E945315CD
:101B10008091440483608093440410924504809132
:101B2000E804873009F487C08830B0F5823009F4C2
:101B300076C0833008F045C0882309F476C0813030
:101B400009F470C00E94531580914C04882359F009
:101B500080914C04815080934C040E947F048091BA
:101B60004C048823A9F70E947829882379F680916C
:101B7000E804863039F781E00E94BA13882311F314
:101B800080E00E948E138823E9F20E94B4160E941E
:101B90001418E0E0F0EF19948C3009F449C08D304E
:101BA00038F4883009F18B3069F60E94FB22AECF01
:101BB0008E30B9F08E3080F18F3021F60E944D2E9C
:101BC000A5CF843059F0843030F0853009F0BACF99
:101BD0000E9439349BCF0E94902598CF0E949D1D72
:101BE00095CF0E94FD1992CF0E94B4160E94531502
:101BF00080914C04882359F080914C04815080934B
:101C00004C040E947F0480914C048823A9F70E9411
:101C10007829882359F37ACF0E94DA4677CF0E9439
:101C2000523E74CF0E94714071CF0E941A126ECF43
:101C30000E9494106BCF0E94492768CF772767FDD9
:101C40007095872F972F22EE34E040E050E00E94FD
:101C5000174860537D4E8C4E9F4FE4CE8CE00E941F
:101C60008E13882309F430CF6E010894C11CD11C57
:101C7000FF24B1E1AB2EB12CAC0EBD1EAFE0EA2EBD
:101C800086010E94F800F801908381830E5F1F4F48
:101C90000A151B05B1F7F60104C031960E171F0790
:101CA00089F02081822F90E08F7090700D9724F042
:101CB000822F8F708083282F2D3079F78E2F8C19EB
:101CC0008F3099F480E060E04F2D21E086010E9482
:101CD000292D85E50E94C9190E941418F394F0E893
:101CE000FF1671F60E94B416EFCEE082D6CF1092A6
:101CF0003C04109279046091790470E06170707016
:101D000062957295707F7627607F762782E090E0FB
:101D10000E9468020E94AE2D1092C0041092AD0481
:101D200083E090E060E00E94680284E090E06091CF
:101D3000AD040E94680288E790E090938C04809341
:101D40008B0485E090E068E770E00E94720280E119
:101D5000809300026091000287E090E00E94680298
:101D60001092A70488E08093AA048091AA0460914D
:101D7000A70490E0019782959295907F9827807FA5
:101D80009827682B8AE090E00E9468028DE090E03E
:101D900060E00E946802F89480ED92E1A3E1B0E077
:101DA0008093090290930A02A0930B02B0930C0255
:101DB000789410E082E20E94711683E20E9471160C
:101DC0000E94141882E30E94E90E1F5F183291F7F7
:101DD00089CF20EA3FE0E22FF32F3197F1F78A9580
:101DE000D1F70895882309F41EC09AEF20EA3FE056
:101DF000E22FF32F3197F1F79A95D1F7E22FF32FD6
:101E00003197F1F79A95D1F7E22FF32F3197F1F748
:101E10009A95D1F7E22FF32F3197F1F79A95D1F7F1
:101E2000815009F0E5CF08951092B6041092BF04D6
:101E300008951F93CF93DF93EC01142F6F7778856C
:101E4000772309F44CC0462F50E0888190E08F77CB
:101E500090704817590779F121E030E00DC0D901A1
:101E6000FE01E20FF31F808190E08F7790702F5F6B
:101E70003F4F8417950709F1271788F3272F2F5F06
:101E8000293030F128E0922F822F9150FE01E80F87
:101E9000F11DDE01A90FB11D8C918083892F99233B
:101EA000A1F71536C0F480E0862B88832887DF9160
:101EB000CF911F910895A0E0B0E0153670F480E056
:101EC000AC0FBD1F862B8C93DF91CF911F9108958E
:101ED0002223C9F6E6CF80E8E7CF80E8F1CF91E092
:101EE00081E021E0D2CFCF93DF93EC01388533231B
:101EF000B9F06F7770E0888190E08F779070681705
:101F0000790789F0FE0120E008C0818190E08F7799
:101F1000907031966817790739F02F5F2317A8F36F
:101F2000DF91CF91089520E0323068F0922F9F5FCB
:101F3000FE01E20FF11DDE01A90FB11D8C9180831E
:101F4000292F9317A0F331503887DF91CF9108954F
:101F5000282F9091AD048091C00085FFFCCF90693F
:101F60009093C6008091C00085FFFCCF822F8F77B1
:101F70008093C60027FD09C090912F028091C00078
:101F800085FFFCCF9093C600089590912D0280911B
:101F9000C00085FFFCCF9093C6000895282F909134
:101FA000AD048091C00085FFFCCF90689093C6007F
:101FB0008091C00085FFFCCF822F8F778093C60071
:101FC00027FD09C090912F028091C00085FFFCCFB2
:101FD0009093C600089590912D028091C00085FFD6
:101FE000FCCF9093C6000895982F8091C00085FF84
:101FF000FCCF9093C60080E090E008959091520449
:102000008091530420E030E0981711F021E030E097
:10201000C901089590915204809153049817D1F307
:10202000F89490915204E92FF0E0EF53FB4F808138
:102030009F5F90935204909152049F719093520429
:10204000789490E0089590915204809153049817E9
:1020500029F00E940A10482F87FD03C040E0842F1A
:102060000895582F52955F705F30C9F3282F30E0E4
:102070002F7030708091C00490E02817390771F7F5
:1020800050934F04ECCF9091AD048091C00085FF38
:10209000FCCF906B9093C6008091C00085FFFCCF71
:1020A0008BE78093C6008091C00085FFFCCF109223
:1020B000C600089580913C04823049F08091C000B0
:1020C00085FFFCCF8CEF8093C6000E9443100895DB
:1020D00090913E048913089580E00E94951D8FEF32
:1020E00080933E0408951F93182F962F6623B9F00E
:1020F00060E080913E048F3F09F061E0953648F43E
:10210000812F895140E00E947E1D10933E041F9153
:102110000895812F895141E00E947E1DF6CF60E035
:102120000E9468101F910895FF920F931F93809152
:10213000980581708093980580919805809381041B
:102140000E94B41680919805882309F032C10E943C
:1021500014188BE090E00E946102809330028CE0C2
:1021600090E00E94610280933102FF2410E00E94FF
:1021700053150E944E0C0E947829882309F04AC00A
:102180009091520480915304981769F00E940A10AC
:10219000682F87FD6DC080914F04883009F4AEC070
:1021A000893009F479C0112371F42091B6042223F7
:1021B00049F48091BF04882329F48091250788235E
:1021C00009F4E2C010E087E10E94E313882379F26A
:1021D000809198058F5F8093980580919805817014
:1021E00080939805809198058093810480E00E94F7
:1021F0003D1680919805882309F4B9CF80E00E94AC
:1022000005160E9453150E944E0C0E9478298823BF
:1022100009F4B6CF0E94431081E080933A06809182
:1022200018078093AB0510923B068091D70660910A
:1022300018074091340620913A060EE716E00E94F6
:10224000B42C60913406C8010E94ED29FF2061F092
:102250008BE090E0609130020E9468028CE090E098
:10226000609131020E9468021F910F91FF900895C2
:10227000482F42954F704F3009F498C0282F30E016
:102280002F7030708091C00490E02817390709F44E
:102290008DC010924F046BCF67FDBAC0062F0E940D
:1022A0000A10482F112309F08ECF509130020517E4
:1022B00048F0852F90E00F96202F30E0821793078B
:1022C0000CF082C050913102051708F46ECF852FB3
:1022D00090E00C96202F30E0821793070CF465CF26
:1022E000051B87EB94E0602F0E94190F8091B704C3
:1022F0008F778093C6062091B60459CF67FD84C0BE
:10230000062F0E940A10112371F540913002041724
:1023100048F0842F90E00F96202F30E0821793072B
:102320000CF06BC040913102041708F43ECF842FAB
:1023300090E00C96202F30E0821793070CF435CFF5
:10234000041B87EB94E0602F0E94730F8091BF0401
:10235000882309F42ACF8091B7048F778093C6062B
:102360002091B60424CF113009F456C089E10E94AF
:102370003D1600933102809198058093810420914D
:10238000B604FF24F39413CF84E00E94E313882360
:10239000A1F485E00E94E313882309F413CF10927F
:1023A000810489E10E94051612E00DCF40934F048D
:1023B000F2CE80E00E940516CACE1092810480E21F
:1023C0000E94051611E0FFCE051B8EEA94E0602FF7
:1023D0000E94190F2091B604209350048091AE04FE
:1023E0008F77809351048091ED04909151048295F0
:1023F000807F890F80935104DACE041B8EEA94E02B
:10240000602F0E94730FE6CF0E940A10082F79CF29
:102410000E940A10082F43CF80E20E943D160093CD
:10242000300280919805809381042091B604FF24A6
:10243000F394BDCE1F930E94C9168091C0040E94E0
:10244000D7160E94531584E60E94E90E0E94531588
:1024500084E60E94E90E0E9453158FEF80933E049C
:102460000E9453150E944E0C0E947829882311F572
:102470009091520480915304981791F30E940A108E
:10248000482F87FD1BC080914F04883049F1893067
:1024900039F747FD32C0142F0E940A10682F812F90
:1024A0000E9473100E9453150E944E0C0E947829BE
:1024B0008823F1F20E9443101F910895582F5295DE
:1024C0005F705F30B9F0282F30E02F70307080914E
:1024D000C00490E02817390769F010924F04C0CF6C
:1024E00047FD0FC0142F0E940A10682F812F0E94F1
:1024F0006810B6CF50934F04C6CF0E940A10182F11
:10250000CBCF0E940A10182FEECF1F920F920FB65A
:102510000F920BB60F9211242F933F934F935F931B
:102520006F937F938F939F93AF93BF93EF93FF939B
:102530009091C6009A3F09F442C09C3FA9F1983F90
:1025400009F44AC080915304E82FF0E0EF53FB4FA9
:1025500090838F5F80935304809153048F71809395
:1025600053049091530480915204981751F4809130
:1025700052048F5F80935204809152048F71809334
:102580005204FF91EF91BF91AF919F918F917F91F5
:102590006F915F914F913F912F910F900BBE0F90D4
:1025A0000FBE0F901F90189580918104882349F3E6
:1025B00080913C04823029F70E940C2EE2CF80915A
:1025C0003C048230F1F680918104882311F00E944E
:1025D00052320E948900D5CF809186049091870461
:1025E00090933A04809339041092870410928604E1
:1025F00080913C04823029F68091390490913A040C
:1026000096958795909356048093550481E0809326
:102610004D0480914C048F5F80934C04B2CF809125
:102620003C04813009F05F98089599B1991F99276A
:10263000991F80915704882311F4992321F49093D2
:10264000570480E008959093570481E0089599B16C
:10265000991F9927991F80915804882311F0992375
:1026600021F09093580480E008951092580481E07E
:1026700008958AB1806F8AB98BB18F708BB9089534
:102680008AB18F708AB98BB18F708BB908958091A0
:102690003C04882321F45C9881E00E94E90E5F9A53
:1026A0000895AC01F8942898000000000000000094
:1026B000289A20E030E01EBC0DB407FEFDCF8EB599
:1026C000FA01E20FF31F80832F5F3F4F2330310564
:1026D00091F77894089516980895169A089520B160
:1026E000269526952F70822F90E02695322F3695CD
:1026F00036952270322B880F991F282F2470322B89
:10270000880F991F880F991F8870382B8FE0831BC3
:10271000089580B1869586958F700895282F883109
:1027200088F4E82FE695E695E695F0E0E251FB4F58
:10273000808190E0277002C0959587952A95E2F7F1
:102740008170089580E00895282F883188F4E82F5B
:10275000E695E695E695F0E0EB51FB4F808190E041
:10276000277002C0959587952A95E2F781700895A4
:1027700080E00895282F883188F4E82FE695E695C3
:10278000E695F0E0E751FB4F808190E0277002C0B2
:10279000959587952A95E2F78170089580E00895D0
:1027A0008091EE04882321F48091EF04882319F0AE
:1027B00090E0892F089590E08091F0048823C9F774
:1027C00091E0892F0895282F8831A0F4482F46954D
:1027D00046954695277081E090E0382F01C0330F71
:1027E0002A95EAF7A42FB0E0FD01EB51FB4F808161
:1027F000832319F420E0822F0895232F30E02095C1
:102800003095A251BB4F8C9190E028233923232B84
:1028100089F7342F3F5F832F63E00E943648E92F0A
:10282000F0E0E251FB4F8081882321F720E0832FE5
:102830008F5F0E943648E92FF0E0E251FB4F808124
:102840008823C9F621E0D7CF1F93CF93DF93C4E449
:10285000D2E010E088810E948E13882329F41F5F44
:1028600021961D30B9F71FEF812FDF91CF911F9176
:1028700008951F93CF93DF93C4E4D2E010E08881E2
:102880000E94A413882349F41F5F21961D30B9F7D5
:1028900080E0DF91CF911F910895812F8F5FDF91AD
:1028A000CF911F9108951F93CF93DF93C4E4D2E09B
:1028B00010E088810E94BA13882349F41F5F219693
:1028C0001D30B9F780E0DF91CF911F910895812FDE
:1028D0008F5FDF91CF911F9108951F93CF93DF9367
:1028E000CCE3D2E010E088810E948E13882349F463
:1028F0001F5F21961830B9F780E0DF91CF911F91CB
:102900000895812F8F5FDF91CF911F9108951F93BD
:10291000CF93DF93CCE3D2E010E088810E94A41330
:10292000882349F41F5F21961830B9F780E0DF91C2
:10293000CF911F910895812F8F5FDF91CF911F91CC
:1029400008951F93CF93DF93CCE3D2E010E088810A
:102950000E94BA13882349F41F5F21961830B9F7F3
:1029600080E0DF91CF911F910895812F8F5FDF91DC
:10297000CF911F910895CF93DF93CCE3D2E088816C
:102980000E948E13882349F4219682E0C434D8072C
:10299000B1F780E0DF91CF91089581E0DF91CF9191
:1029A0000895FF920F931F93CF93DF93CCE3D2E070
:1029B000FF2400E006C00F5F219682E0C434D807F0
:1029C00089F01881812F0E948E138823A1F7812F0F
:1029D0000E94BA13882381F3F394219682E0C434D1
:1029E000D80779F781E0F81639F080E0DF91CF91D0
:1029F0001F910F91FF90089580E00730B9F781E0B3
:102A0000F5CF1F93CF93DF93C2E3D2E010E088812C
:102A10000E94A413882349F41F5F21961A30B9F746
:102A200080E0DF91CF911F910895812F8F5FDF911B
:102A3000CF911F91089580915A0410925A040895DD
:102A400080E00895382F883100F5282F277081E025
:102A500090E0982F01C0990F2A95EAF7832F869569
:102A600086958695A82FB0E0FD01EB51FB4F808144
:102A7000892369F4FD01E751FB4F8081892371F4BB
:102A8000A251BB4F8C91982339F480E00895832F95
:102A90000E94E31882E0089583E00895832F0E9446
:102AA000EB1881E00895EF92FF920F931F93DF934D
:102AB000CF9300D000D0CDB7DEB71092E5041092CE
:102AC000E9041092E6041092EA041092E7041092CE
:102AD000EB0480915B048A3068F426960FB6F89474
:102AE000DEBF0FBECDBFCF91DF911F910F91FF9041
:102AF000EF90089510925B0416987E010894E11CF3
:102B0000F11CC7010E9451138091EE048C838091C7
:102B1000EF048D838091F0048E8360E070E001E02B
:102B200010E0E62FE695E695E695F0E0CB0187709C
:102B30009070980102C0220F331F8A95E2F7C901F5
:102B4000AF0142515B4FD701AE0FBF1F3C91EF5019
:102B5000FB4F2081232B28238095FA01308183238A
:102B6000282B20836F5F7F4F68317105D1F60E945B
:102B70006F13982F96959093ED048093E304169A23
:102B800040E050E0BE016C5F7F4FDA01AF50BB4FB9
:102B9000F701E40FF51F80818C93FB01E40FF51F13
:102BA0002081FA01E251FB4F9081FA01EB51FB4F7A
:102BB000822F809589238083FA01E751FB4F9095FE
:102BC000922390834F5F5F4F43305105F1F690B1F0
:102BD000969596959F708091E104891721F0109247
:102BE0005C049093E10480915C048F3630F0909304
:102BF000E2048091E2048093E10482E00E948E135B
:102C000080934B040E94141868CF282F8832C0F498
:102C1000E82FE695E695E695F0E0277081E090E0F4
:102C200001C0880F2A95EAF7DF01A35ABB4F2C9108
:102C3000282B2C93EE59FB4F809520818223808393
:102C40000895282F8832C0F4E82FE695E695E6959A
:102C5000F0E0277081E090E001C0880F2A95EAF744
:102C6000DF01AE59BB4F2C91282B2C93E35AFB4F1D
:102C700080952081822380830895282F8832C8F48C
:102C8000E82FE695E695E695F0E0277081E090E084
:102C900002C0880F991F2A95E2F78095DF01A35A99
:102CA000BB4F2C9128232C93EE59FB4F208182237C
:102CB00080830895282F883298F4E82FE695E695CA
:102CC000E695F0E0EE59FB4F277081E090E002C0FE
:102CD000880F991F2A95E2F78095208182238083AF
:102CE0000895282F883290F4E82FE695E695E6952A
:102CF000F0E0E35AFB4F277081E090E002C0880FBC
:102D0000991F2A95E2F72081282720830895E82F2C
:102D1000883298F4282F277081E090E002C0880F55
:102D2000991F2A95E2F7E695E695E695F0E0EE59CB
:102D3000FB4F20812823822F089520E0822F0895C1
:102D4000982F969596959695EDE5F4E0E90FF11D8F
:102D5000208130E0877002C0359527958A95E2F78B
:102D600021703070C90108951092610410926004BE
:102D700010925F0410925E0410925D04109266043B
:102D8000109265041092640410926304109262041D
:102D90000895CF93DF93C0EBD2E089910E943D1656
:102DA00082E0C03CD807C9F7DF91CF910895803108
:102DB00008F00895E82FF0E0E055FD4F80810E9473
:102DC00005160895803108F00895E82FF0E0E055E9
:102DD000FD4F80810E943D1608950F931F93CF935E
:102DE000DF93082FC0EBD2E010E007C088810E947B
:102DF00005161F5F2196103149F01017B8F388812E
:102E00000E943D161F5F21961031B9F7DF91CF91D7
:102E10001F910F910895803108F00895E82FF0E098
:102E2000E055FD4F80810E9421160895803110F0F9
:102E300080E00895E82FF0E0E055FD4F80810E948A
:102E4000A0160895803110F080E00895E82FF0E09A
:102E5000E055FD4F80810E9487160895883108F063
:102E60000895E82FF0E0E557FD4F80810E94051698
:102E70000895883108F00895E82FF0E0E557FD4FF8
:102E800080810E9421160895883108F00895E82F66
:102E9000F0E0E557FD4F80810E943D160895CF93E5
:102EA000DF93CBE8D2E089910E943D1682E0C33ADD
:102EB000D807C9F7DF91CF910895E82F8150883066
:102EC00008F00895F0E0EE57FD4F80810E9405164E
:102ED00008950F931F93CF93DF93082FC3E8D2E099
:102EE00011E007C088810E943D161F5F21961930AE
:102EF00069F01017B9F7E12FF0E0EE57FD4F808130
:102F00000E9405161F5F2196193099F7DF91CF9126
:102F10001F910F910895E82F8150883008F008958F
:102F2000F0E0EE57FD4F80810E943D160895E82F96
:102F30008150883008F00895F0E0EE57FD4F808111
:102F40000E9421160895E82F8150883010F080E00B
:102F50000895F0E0EE57FD4F80810E948716089596
:102F6000E82F8150883010F080E00895F0E0EE57AF
:102F7000FD4F80810E94A0160895CF93DF93C3E890
:102F8000D2E089910E943D1682E0CB38D807C9F77C
:102F9000DF91CF9108958D3008F00895E82FF0E08B
:102FA000ED55FD4F80810E94051608958D3008F083
:102FB0000895E82FF0E0ED55FD4F80810E943D1609
:102FC00008958D3008F00895E82FF0E0ED55FD4F9D
:102FD00080810E9421160895E3EAF2E0E80FF11DD6
:102FE00080810E9487160895CF93DF93C3EAD2E0D1
:102FF00089910E943D1682E0C03BD807C9F7DF9156
:10300000CF9108950E94F41784E00E943D1683E05A
:103010000E943D1688E00E943D1681E00E943D1608
:1030200082E00E943D160895F894179820E030E061
:1030300090916704F901EE59FB4F80819823F901C3
:10304000E35AFB4F8081982B9EBD0DB407FEFDCF48
:103050002F5F3F4F2530310559F7179A789408951F
:10306000EDE5F4E0A2E6B4E080819D91892B8193A7
:1030700084E0E236F807C1F70895EDE5F4E0A2E652
:10308000B4E09D91909580818923819384E0E2361C
:10309000F807B9F70895EDE5F4E0A2E6B4E0208181
:1030A0009C91892F822319F09095922390831D92F1
:1030B000319684E0E236F80791F708951F93182FB0
:1030C00084E00E943D16123049F083E00E943D16D4
:1030D000113071F01F3F39F01F91089583E00E9475
:1030E00021161F91089584E00E9405161F910895EE
:1030F00083E00E9405161F9108950F931F93CF93AD
:10310000DF93182F87FD50C086E10E944417812F5E
:10311000829586958695837080FF29C085E10E94FF
:103120002E171F7349F11731A0F58FEF0E945E181B
:1031300084E10E944417012F10E0CBE0D0E0C017DB
:10314000D10731F0FE01E856FD4F80810E943D1607
:103150002196C831D10599F708561D4FF801808195
:103160000E940516DF91CF911F910F91089585E17F
:103170000E9444171F73B9F680E00E945E180E94F7
:10318000F41784E10E942E17DF91CF911F910F91C8
:103190000895143268F0103370F4185181E00E94E1
:1031A0005E18112329F6EBCF86E10E942E17AFCFD0
:1031B0001C5080E0F4CF1C3318F4145282E0EFCF9F
:1031C000105383E0ECCFEBE8F2E0E80FF11D8081D3
:1031D0000E9405160895EBE8F2E0E80FF11D8081EA
:1031E0000E943D160895E3E8F2E0E80FF11D8081AA
:1031F0000E9405160895E3E8F2E0E80FF11D8081D2
:103200000E943D160895DF92EF92FF920F931F9355
:10321000CF93DF93F02EDE2C222371F1022F040FC7
:10322000E42EC3E8D2E010E00BC0101758F41F15CD
:10323000D9F088810E9405161F5F2196183049F049
:103240001E1598F788810E943D161F5F2196183041
:10325000B9F781E08D15A0F4DF91CF911F910F9107
:10326000FF90EF90DF900895E12FF0E0ED57FD4FD4
:1032700080810E942116E0CF062F080FE82ED1CFC3
:10328000DD2071F088E00E943D1681E00E94051665
:10329000DF91CF911F910F91FF90EF90DF900895F4
:1032A00088E00E94051681E00E943D16DF91CF91D3
:1032B0001F910F91FF90EF90DF900895FF920F9371
:1032C0001F93082FF62E84E00E943D1683E00E9493
:1032D0003D1688E00E943D1681E00E943D16102FA9
:1032E00004FD34C015FD29C007FD2CC016FD21C00A
:1032F0000E94F417FF2099F0802F8F708D3098F086
:103300008BE10E9405168CE10E9405168FE00E9459
:1033100005168EE00E9405168DE00E9405161F918D
:103320000F91FF9008950E94CB171F910F91FF906E
:10333000089581E00E940516DBCF83E00E94051608
:1033400007FFD4CF88E00E940516D0CF84E00E940A
:103350000516C8CFE1E5F2E0E80FF11D8081089580
:103360008A3008F00895E82FF0E0E758FD4F80819B
:103370000E9405160895CF93DF93C9E7D2E08991A3
:103380000E943D1682E0C338D807C9F7DF91CF917C
:10339000089590915D04982790935D0490915E0448
:1033A000982790935E0490915F04982790935F0410
:1033B00090916004982790936004909161049827FD
:1033C000909361040895AC0161157105A1F020E0AE
:1033D000E0E0A0E0B0E0A40FB51F8C91E827F0E09A
:1033E000E853FD4FE0812F5FA22FB0E0A617B7078B
:1033F00090F38E2F0895E0E0FCCF0E9453150E94B9
:103400004E0C0E9478298823C1F30895EF92FF9211
:103410000F931F93CF93DF937C018B01611571058F
:1034200061F0C0E0D0E0F701EC0FFD1F80810E9449
:10343000E6012196C017D107B0F3DF91CF911F911C
:103440000F91FF90EF90089522E42093F4041092DE
:10345000F50422E02093F6049093F7048093F80497
:10346000A4EFB4E0E0E08D91E827F0E0E853FD4FF1
:10347000E08184E0A93FB807B1F7EC93CD0105974F
:1034800066E070E00E94061A089590E89093F404B4
:103490001092F50421E02093F6048093F704A8EC41
:1034A000B2E090914803FD01E90FF11D9081922750
:1034B000FD01E90FF11D90819827A90FB11D8C9195
:1034C0008093F80484EF94E065E070E00E94061AAF
:1034D00008951F920F920FB60F920BB60F92112400
:1034E000DF92EF92FF920F931F932F933F934F938F
:1034F0005F936F937F938F939F93AF93BF93CF937C
:10350000DF93EF93FF931091CE008091C702882341
:1035100009F46EC080916A0490916B04895E9340B7
:1035200008F080C080916804803408F089C0282F9A
:103530002F5FE82FF0E0EC5CFA4F108320936804D3
:1035400010926B0410926A04233008F451C07091F9
:1035500034059091350580E060913605462F50E0A6
:10356000482B592B30E0CA0104962817390708F474
:103570003FC09A012D5F3F4FF901EC5CFA4F10817B
:103580002115310509F401C190E0E0E0A0E0B0E0D0
:10359000AC5CBA4F8C91E827F0E0E853FD4FE08136
:1035A0009F5FA92FB0E0A217B30790F31E1709F48D
:1035B00050C02115310509F4EAC090E0E0E0A0E038
:1035C000B0E0AC5CBA4F8C91E827F0E0E853FD4FD7
:1035D000E0819F5FA92FB0E0A217B30790F38E2F71
:1035E00090E00E94C2011092680480E00E94451A97
:1035F000FF91EF91DF91CF91BF91AF919F918F910B
:103600007F916F915F914F913F912F911F910F91FA
:10361000FF90EF90DF900F900BBE0F900FBE0F90BA
:103620001F9018950E94C9160E9414181093340513
:1036300081E08093680410926B0410926A04D8CFE2
:103640000E94451A1092680410926B0410926A044A
:10365000CFCF713809F492C17238B0F5713109F4E5
:103660002BC1723108F096C0713051F1703131F0D8
:1036700080E00E94451A10926804BACF6231C1F707
:1036800080913705082F10E0000F111F000F111F48
:10369000000F111F80913805080F111D029512951A
:1036A000107F1027007F1027C9E3D5E08991B8016A
:1036B0000E94601E0F5F1F4F85E0C934D807B1F725
:1036C00081E00E94451AD7CF763809F435C17738A2
:1036D00008F073C0723809F484C1753849F6433074
:1036E000510509F0A5C030913705932F80E0209156
:1036F0003805E22EFF24E82AF92AD0903905EAE3BA
:10370000ED1508F4B6CF7093F4041092F504F2E0CE
:10371000DF0ED092F6048EEFD80E3093F70420938C
:10372000F804DD2071F009EF14E0E701CE010E94FA
:10373000A41EF80181938F0121969E012E192D154B
:10374000A8F38091F604682F6D5F09F4D5C1A4EF4A
:10375000B4E090E08E5F282F30E02B503B4F8D91EE
:103760009827E92FF0E0E853FD4F9081A217B307A7
:10377000B1F7E62FF0E0EC50FB4F90836F5F84EFE2
:1037800094E070E00E94061A76CFE0E00FCF80E070
:1037900090E027CF703409F453C1713409F068CF39
:1037A000623009F065CF9091370580E020913805AF
:1037B000820F911D0E94CC025ECF7738E9F17838F4
:1037C00009F056CF7093F4041092F50480913705F8
:1037D000813009F46AC1813008F05BC180E18093D7
:1037E000F7041092F8048093F9041092FA0484E02C
:1037F00047E0A7E0B0E068E070E08093F60490E076
:1038000020E030E0F901EC50FB4F80819827E92F50
:10381000F0E0E853FD4F90812F5F3F4F241790F366
:10382000AC50BB4F9C9384EF94E00E94061A23CFC8
:1038300080E00E94451A1FCF80913705882309F048
:1038400006C14230510509F014CFE0913805E4304B
:1038500008F00ECF89E18093F4041092F50480E122
:103860008093F6042E2F30E022953295307F322758
:10387000207F3227A7EFB4E0F901E258F94F8081A9
:103880008D932F5F3F4F85E0A730B807A9F7539777
:10389000E0E08D91E827F0E0E853FD4FE081F5E0AE
:1038A000A730BF07B1F7E0930705CD01439764E167
:1038B00070E00E94061ADFCE623009F0D9CE809106
:1038C0003705082F10E0000F111F000F111F000F08
:1038D000111F80913805080F111D02951295107F58
:1038E0001027007F102789E18093F4041092F504DB
:1038F00080E18093F604C7EFD4E0C8010E94A41EC3
:1039000089930F5F1F4F35E0C730D307B1F7DE0152
:103910005397E0E08D91E827F0E0E853FD4FE08118
:10392000CA17DB07B9F7E093070584EF94E064E179
:1039300070E00E94061A9FCE9091370580E020919A
:103940003805E22EFF24E82AF92A2EEFD22ED60ED1
:1039500063506A3308F06CCFDD2009F4B1CE09E37F
:1039600015E0E701F80181918F01BE010E94601E00
:1039700021969E012E192D15A8F3A2CE87E190E085
:103980009093F8048093F7048DEC90E09093FA0400
:103990008093F904E0ECF2E0ABEFB4E081918D9319
:1039A00022E0E63CF207D1F781E88093F40410921C
:1039B000F5048AE08093F604A4EFB4E0E0E08D9192
:1039C000E827F0E0E853FD4FE08135E0A130B30790
:1039D000B1F7EC93CD010D976EE070E00E94061AEE
:1039E0004ACE4230510509F023CF309137053323B9
:1039F00009F468C09091380520E082E88093F404CF
:103A00001092F50483E08093F6043093F7049093CA
:103A1000F8042093F904A4EFB4E0E0E08D91E827E6
:103A2000F0E0E853FD4FE08184E0AA3FB807B1F72A
:103A3000EC93CD01069767E070E00E94061A1BCE5A
:103A400080918B0490918C040E94241A14CE8130B2
:103A500009F00ECE4231510509F00ACEE091380549
:103A6000E43008F005CE2E2F30E0A9E3B5E0229532
:103A70003295307F3227207F32278D91F901E2582D
:103A8000F94F80832F5F3F4F85E0A934B807A9F72E
:103A900017CE883009F0ECCD81E08093F70444E044
:103AA000A4E0B0E065E070E0A8CE88E08093F70481
:103AB00080E18093F80482E045E0A5E0B0E066E0B4
:103AC00070E09BCE90913805973860F4953870F48B
:103AD000993181F0993120F0892F8158823030F06E
:103AE00020E08BCF973821F09838D1F721E085CFAF
:103AF00024E083CF20E181CF90E03BCE2C9880342E
:103B000008F08FE3611160E4442349F090E08823DA
:103B100049F0682B962B98B92C9A2D9A089590E825
:103B20008823B9F7962B98B90895882319F42D980E
:103B30002C980895469A2C9808959F92AF92BF9220
:103B4000CF92DF92EF92FF920F931F93CF93DF9369
:103B50000E94C9168091AD040E94D7160E94531589
:103B60000E941B15BB249924AA24CC240E9453151F
:103B70000E944E0C0E947829882309F075C02B2DD5
:103B80003CE02302C001112497E1D92ED80EEA2C83
:103B9000E294EE0CEE0C80ECE822C0E0D0E009C02C
:103BA000802F0E94BA13882319F52196CD30D105B4
:103BB00059F1FC2EFE01E853FC4F0081802F0E943A
:103BC000A413882369F31C2F1D0D812F6C2D4A2D02
:103BD0000E947E1D812F8E290E94A80F8C2F0E948B
:103BE000CB17CC24C394802F0E94BA138823E9F208
:103BF0008F2D8D0D8E290E94CE0F8F2D0E94D617EE
:103C00002196CD30D105A9F68FE00E94A413882318
:103C100009F444C081E08B150CF050C09B1429F0CE
:103C20008B2D0E945E180E94141884E10E94A41338
:103C3000882351F080E0AA2009F481E0A82E88238F
:103C4000C9F188E00E94051686B190E08F739070EC
:103C5000892BC1F49B2C0E9453150E944E0C0E948C
:103C60007829882309F48BCF0E944310DF91CF91EC
:103C70001F910F91FF90EF90DF90CF90BF90AF908A
:103C80009F9008950E94D013882321F380E00E9422
:103C9000951D0E94F417CC249B2CDDCF8EE00E9452
:103CA000A413882309F4BACF2FEFB21609F4B6CFC4
:103CB000BA94B4CF88E00E943D16C6CFB394AECF7D
:103CC000282FF89495E028980000000000000000DC
:103CD0009EBD0DB407FEFDCF0000000000000000F7
:103CE0001EBC0DB407FEFDCF8EB5289A0000000063
:103CF0000000000080FDE7CF28980000000086E06B
:103D00008EBD0DB407FEFDCF00000000289A000014
:103D100000000000000028980000000082E08EBD36
:103D20000DB407FEFDCF7EBD0DB407FEFDCF6EBD09
:103D30000DB407FEFDCF2EBD0DB407FEFDCF000074
:103D40000000289A78940895382FF89425E0289850
:103D500000000000000000002EBD0DB407FEFDCFE6
:103D600000000000000000001EBC0DB407FEFDCFE7
:103D70008EB5289A000000000000000080FDE7CF0B
:103D800028980000000083E08EBD0DB407FEFDCF33
:103D90009EBD0DB407FEFDCF3EBD0DB407FEFDCFA9
:103DA000000000001EBC0DB407FEFDCF8EB5289AA2
:103DB00078940895892F8F7184FD806E0895EF9215
:103DC000FF920F931F93FA01D90186958083862F66
:103DD00090E08F70907095958795959587959595BE
:103DE00087958C93862F8770F801808362956F701A
:103DF000F70160831F910F91FF90EF900895FC01F0
:103E000030E022953295307F3227207F3227208381
:103E10008081660F660F660F640F6F70862B80833C
:103E2000089580916C04882349F087FD0EC083E0DB
:103E30000E94051684E00E943D16089583E00E94CA
:103E40003D1684E00E943D16089583E00E943D16D1
:103E500084E00E9405160895962F803110F08FEFB0
:103E60000895682F70E0660F771F6F5F734F892F7B
:103E70000E94601E80E008959B01803120F5682F2C
:103E800070E0FB01EE0FFF1FEB52FC4F8081918130
:103E900028173907A0F0009749F08150660F771F67
:103EA0006050744F0E94601E80E0089580E0660FAD
:103EB000771F6050744F0E94601E80E00895C90112
:103EC000009759F7F3CF8FEF0895803198F470E0A1
:103ED0006050784F90E000249695879507949695CA
:103EE00087950794982F802D680F791F8CE060309C
:103EF000780710F08FEF0895842F0E94601E80E0F5
:103F00000895EF92FF920F931F93CF93DF93C82FE3
:103F1000D0E0CC0FDD1FCC0FDD1FCC0FDD1FC60F97
:103F2000D11DC05CDF4FCC0FDD1FC295D295D07F75
:103F3000DC27C07FDC27EE24FF248701000F111F40
:103F40000C581A4FF80180819181892FBE010E947F
:103F5000601EF801808191812196BE010E94601E41
:103F60000894E11CF11C2196F0E1EF16F10429F709
:103F7000DF91CF911F910F91FF90EF90089590E006
:103F8000880F991F8F5F934F0E94A41E90E00895A1
:103F90000F931F93082F10E0000F111FC8018050CE
:103FA000944F0E94A41E90E001960B521C4FF80102
:103FB000208131818217930708F49C01C9011F9168
:103FC0000F9108958091E3048093A5058091A50544
:103FD0000E94C81F9093A00580939F058091A5051E
:103FE0000E94BF1F9093A7058093A6052091A60568
:103FF0003091A70580919F059091A005281739075A
:1040000020F01092A7051092A6058091940590913A
:104010009505E091A505F0E0EE0FFF1FEB52FC4F78
:10402000608171810E944248909395058093940528
:104030000895803198F470E06050784F90E000244B
:10404000969587950794969587950794982F802D38
:10405000680F791F8CE06030780710F08FEF0895BB
:10406000CB010E94A41E0895EF92FF920F931F931D
:10407000CF93DF93E0909405F09095050894E11CB0
:10408000F11C80E00E94E3138823C9F400E08091D2
:10409000A805813029F180E00E94BA13882329F015
:1040A0008091A805882309F0BFC0013009F4E7C05A
:1040B000DF91CF911F910F91FF90EF90089581E0D4
:1040C0008093A8051092A4051092A3058093730411
:1040D00082E20E943D1601E08091A8058130D9F668
:1040E0000E940115282F8823B9F021508091A30543
:1040F0009091A4057C01EE0CFF1CEE0CFF1CEE0C55
:10410000FF1C880F991FE80EF91EE20EF11CF092B9
:10411000A405E092A30501E087E10E94A41388238F
:1041200041F0E090A605F090A7050894E11CF11C71
:1041300001E083E00E94A413882329F0E0909F050A
:10414000F090A00501E089E00E94A413882309F003
:10415000A2C089E00E94BA13882309F0BAC08AE09D
:104160000E94A413882309F0A5C08AE00E94BA1314
:10417000882309F490CF8CE10E943D16E091A505BB
:1041800020919F053091A005F0E0EE0FFF1FEB524C
:10419000FC4F808191812817390708F07CCF8091EE
:1041A0009F059091A00501969093A00580939F058F
:1041B0008091A50560919F057091A0050E943C1F0C
:1041C0008091A5050E94C81F9093A00580939F052C
:1041D00060919F057091A005615070408091940599
:1041E0009091950586179707D8F4EB01219701C0A8
:1041F000E9018091A5051C2F6C2F0E941920482FE2
:104200008091A5051F5F612F0E94651F9E012150AF
:10421000304080919405909195058C179D0740F34F
:1042200088E08093760437CF82E20E9405161092D0
:1042300073041092A80581E0809376042091A30571
:104240003091A40521153105A9F0E091A505F0E014
:10425000EE0FFF1FEB52FC4F808191818217930775
:1042600048F021503040309395052093940587E025
:104270008093760410924604013009F019CFC701EB
:104280000E94030200934604DF91CF911F910F918A
:10429000FF90EF9008958BE10E9405161092A405FF
:1042A0001092A305E0909405F09095050894E11C08
:1042B000F11C4FCF8CE10E9405161092A4051092BC
:1042C000A305E0909405F09095050894E11CF11C7D
:1042D0004CCF8BE10E943D16C0919405D09195057D
:1042E000219680919F059091A005C817D90708F0E5
:1042F00036CF8091A5051C2F6C2F0E941920482FC6
:104300008091A5051150612F0E94651F2196809113
:104310009F059091A005C817D90758F380919F0574
:104320009091A00501979093A00580939F0580919F
:10433000A50560919F057091A0050E943C1F80918A
:10434000A5050E94C81F9093A00580939F0588E053
:104350008093760404CFEF92FF920F931F93809186
:10436000E3048093A5058091A5050E94C81F909342
:10437000A00580939F058091A5050E94BF1F909383
:10438000A7058093A6052091A6053091A7058091E9
:104390009F059091A0052817390720F01092A705D6
:1043A0001092A6058091940590919505E091A50540
:1043B000F0E0EE0FFF1FEB52FC4F608171810E9415
:1043C000424890939505809394058091A50560914E
:1043D0009405709195050E94192080939C05809109
:1043E000A50560919C0543EF55E02BEA35E00DEA09
:1043F00015E0EFEBEE2EE6E0FE2E0E94DF1E81E0E0
:1044000080933B060E94A9298091BF068093C6062F
:104410001F910F91FF90EF900895AF92BF92CF92AE
:10442000DF92EF92FF920F931F93CF93DF93C82EEB
:10443000DD24CC0CDD1CCC0CDD1CCC0CDD1CC60E34
:10444000D11C80E490E0C80ED91ECC0CDD1CC294B7
:10445000D29410EFD122DC24C122DC24AA24BB2474
:10446000C6010E94A41ED82FC0E07501EE0CFF1CEF
:10447000E4E7F5E0EE0EFF1EF701D183C083008173
:104480001181C60101960E94A41E90E0082B192BF1
:10449000F701118300830894A11CB11C82E090E015
:1044A000C80ED91E90E1A916B104D1F6DF91CF91C3
:1044B0001F910F91FF90EF90DF90CF90BF90AF9042
:1044C000089510929E0584E20E943D160E94B41643
:1044D0000E944B181092390680E00E94951D0895A5
:1044E00010929D05109239061092960580E00E9468
:1044F000951D0E94B4160E944B180E941B1508952A
:1045000080919A0590919B05682F67709695879585
:1045100096958795969587958F700E94762D6091D8
:104520009A0570919B059B0140E050E0DA01C901BA
:1045300080709078A070B070892F9A2FAB2FBB2716
:1045400080937D04DA01C90180709074A070B0700E
:10455000892F9A2FAB2FBB2780937B04207030725A
:1045600040705070232F342F452F552720937C0403
:104570001092AE05872F8F7184FD806E089581E0C3
:1045800080939D0581E20E94051610927B04809124
:104590007B0480937C0480917C0480937D04109242
:1045A0009605109239068091740590917505909347
:1045B0009B0580939A058F5F9F4F89F01092A2050B
:1045C0001092AE05109289040E94802280936C04A0
:1045D00080913D0480FDFCCF81E0809396050E9490
:1045E000C916089581E080939E0584E20E94051615
:1045F0000E94C9160895DF92EF92FF920F931F93C6
:1046000080912507882309F487C284E00E942D2A1F
:104610001092990580919905809398051092A805AC
:104620001092A4051092A3050E94AB218091D70699
:10463000609118074091340620913A060EE716E083
:104640000E94B42C8091340660913A064091AD05E9
:1046500020913B060091B105E090AB050E94031943
:1046600057E0D52E07C0113009F4FFC00E944B2C33
:104670008823D9F00E9453150E944E0C1091BE065B
:104680001330E9F0143078F31430E9F11D3071F78C
:1046900081E00E949D328091BE068D3039F31092E8
:1046A00081040E944B2C882329F70E941A2C0E9417
:1046B00053150E944E0C1091BE06133019F70E943C
:1046C000332A882309F09EC10E94A52B882321F05C
:1046D00010927304109281040E943914882331F2DD
:1046E000182F11500E94F417812F0E94CB1710939E
:1046F000BF0680912507882309F0B8CF8091BF06B7
:104700008093C606B3CF0E94332A882309F05CC188
:104710008091A805882309F44AC10E94342083E0CF
:104720000E94E313882309F03BC187E10E94E31351
:10473000882309F02EC186E10E94E313882309F43F
:1047400068C080913B06882309F0B0C18091BF0604
:104750008093C606E0909405F090950580919905A8
:10476000882309F090C180913A06882309F44AC051
:1047700010E020911807309134068091C60690E031
:1047800082959295907F9827807F982780939C05AB
:1047900080919C05220F220F220F230F210F2F70D3
:1047A000282B20939C058091A5056091940570911C
:1047B000950540919C050E94651F1F5F809194059F
:1047C0009091950501969093950580939405089492
:1047D000E11CF11C8091940590919505E091A5054F
:1047E000F0E0EE0FFF1FEB52FC4F608171810E94E1
:1047F0004248909395058093940580913A06181746
:1048000008F4B7CF80919805882309F052C1D0925F
:10481000760480917604873009F407C1809176048C
:10482000883009F459C180917604813009F4AEC012
:104830008091BE06843011F010928104809125078A
:10484000882309F4DBC080918004813009F00ECF09
:10485000109280040E947829882309F407CF1F91C1
:104860000F91FF90EF90DF9008950E94332A8823E4
:1048700009F073C00E94342083E00E94E313882370
:1048800039F583E00E94BA138823F1F49091A505CD
:104890008091E304981711F00E94AB218091BE062D
:1048A000813011F01092810480912507882309F04E
:1048B000B8C00E947829882309F4D8CE1F910F919F
:1048C000FF90EF90DF90089583E20E943D16DECFC7
:1048D00010929505109294058091A505609194051C
:1048E000709195050E94192080939C058091A505E3
:1048F00060919C0543EF55E02BEA35E00DEA15E0A9
:10490000AFEBEA2EA6E0FA2E0E94DF1E81E0809334
:104910003B068091BF068093C6060E94A92980911C
:10492000D706609118074091340620913A060EE7A9
:1049300016E00E94B42C8091340660913A064091B2
:10494000AD0520913B060091B105E090AB050E94BA
:10495000031983E20E94051694CF0E94B41682E2E6
:104960000E9405161093810481E20E943D168091F9
:10497000340660913A064091AD0520913B060091C6
:104980003406E090AB050E94031974CF10927604B0
:104990004FCF81E08093990580E00E942116CBCE15
:1049A00081E08093980583E20E942116BECE0E948A
:1049B000382C9091A50596959093ED04882309F0E5
:1049C000ACCE0E949D32A9CE0E94B41682E20E9413
:1049D000051681E08093810481E20E940516809192
:1049E000340660913A064091AD0520913B06009156
:1049F0003406E090AB050E9403198ACE81E00E9444
:104A00002D2A21CF0E94B41611E01093730484E282
:104A10000E9405168091BF060E94CB171093810457
:104A200053CE84E00E942D2A44CF8091A505609149
:104A30009405709195050E94192080939C058091A2
:104A4000A50560919C0543EF55E02BEA35E00DEAA2
:104A500015E09FEBE92E96E0F92E0E94DF1E11E093
:104A600010933B068091340660913A064091AD0563
:104A700020913B060091B105E090AB050E9403191F
:104A800010937604D0CE109299058091A5056E2DD5
:104A90000E942C1F8091A5050E94BF1F9093A7051F
:104AA0008093A60580E00E943D165DCE0E94A92954
:104AB0004DCE109298058091A505B7010E943C1F2C
:104AC0008091A5050E94C81F9093A00580939F0523
:104AD00083E20E943D169BCE8091A50560919405CE
:104AE000709195050E94192080939C058091A505E1
:104AF00060919C0543EF55E02BEA35E00DEA15E0A7
:104B0000BFEBEB2EB6E0FB2E0E94DF1E81E0809310
:104B10003B061092760487CE81E00E942D2A78CD44
:104B2000EF92FF920F931F9380912507882309F43A
:104B3000ACC184E00E942D2A1092990580919905BC
:104B4000809398051092A8051092A4051092A305D1
:104B50000E94AB218091D7066091180740913406DE
:104B600020913A060EE716E00E94B42C809134069C
:104B700060913A064091AD0520913B060091B10548
:104B8000E090AB050E94031908C0143009F461C01D
:104B90000E944B2C882309F492C00E9453150E9456
:104BA0004E0C1091BE06113081F70E94332A8823E3
:104BB00009F0DAC083E00E94E313882309F0F5C00E
:104BC00083E00E94BA13882309F039C180E00E9473
:104BD000E313882309F03CC180E00E94BA138823C4
:104BE00009F04BC19091A5058091E3049817E1F07D
:104BF0000E94AB218091D70660911807409134063E
:104C000020913A060EE716E00E94B42C80913406FB
:104C100060913A064091AD0520913B060091B105A7
:104C2000E090AB050E9403198091BE06813011F01F
:104C30001092810480912507882309F043C00E94C7
:104C40007829882309F4A4CF1F910F91FF90EF904A
:104C500008950E94332A882309F065C086E10E94E6
:104C6000E313882309F053C083E00E94E3138823F1
:104C700009F041C080E00E94E313882339F580E009
:104C80000E94BA13882379F58091BE06843011F012
:104C90001092810480912507882309F461C08091D6
:104CA0008004813009F074CF109280040E9478292A
:104CB000882351F60E944B2C882309F06ECF0E9466
:104CC0001A2C6BCF84E00E942D2AB9CF11E01093EB
:104CD000A80582E20E943D161093460480E00E94DF
:104CE000BA13882389F282E20E9405161092A80561
:104CF00010924604C9CF81E08093980583E20E9418
:104D000005161092990580E00E943D16B3CF81E010
:104D10008093990580E00E9405161092980583E221
:104D20000E943D16A1CF0E94B41682E20E94051691
:104D300081E08093810481E20E940516809134060F
:104D400060913A064091AD0520913B0600913406F2
:104D5000E090AB050E94031981E00E943F027ECFE4
:104D600081E00E942D2A9BCF0E94B41682E20E940D
:104D700005161093810481E20E943D16809134064D
:104D800060913A064091AD0520913B0600913406B2
:104D9000E090AB050E94031981E00E943F0283E08E
:104DA0000E94E313882309F40BCF1092950510920B
:104DB00094058091A50560919405709195050E94D8
:104DC000192080939C058091A50560919C0543EF77
:104DD00055E02BEA35E00DEA15E07FEBE72E76E0B3
:104DE000F72E0E94DF1E81E080933B068091BF0674
:104DF0008093C6060E94A9298091D7066091180762
:104E00004091340620913A060EE716E00E94B42C39
:104E10008091340660913A064091AD0520913B06A1
:104E20000091B105E090AB050E94031983E20E9456
:104E3000051683E00E94BA13882309F4C7CE83E2E3
:104E40000E943D1680E00E94E313882309F4C4CE3B
:104E500011E01093A80582E20E943D16809194050E
:104E60009091950501960E9403021093460480E0FC
:104E70000E94BA13882309F4B5CE82E20E94051677
:104E80001092A80510924604ADCE81E00E942D2A12
:104E900053CEEF920F931F9310926E0480912507CB
:104EA000882309F421C284E00E942D2A10929905DA
:104EB00080919905809398051092A8051092A405F9
:104EC0001092A3050E94E21F07C0113009F493C09D
:104ED0000E944B2C8823D9F00E9453150E944E0C3F
:104EE0001091BE061330E9F0143078F31430E9F174
:104EF0001D3071F781E00E949D328091BE068D3099
:104F000039F3109281040E944B2C882329F70E94C8
:104F10001A2C0E9453150E944E0C1091BE0613309D
:104F200019F70E94332A882309F0B0C00E94A52BEC
:104F3000882321F010927304109281040E94391486
:104F4000882331F2182F11500E94F417812F0E94EC
:104F5000CB171093BF0680912507882309F0B8CF9F
:104F60008091BF068093C606B3CF0E94332A882360
:104F700009F0D5C08091A805882309F4C3C083E057
:104F80000E94E313882329F080916E04813009F494
:104F900087C187E10E94E313882309F08CC080E079
:104FA0000E94E313882309F092C080E00E94BA13A4
:104FB000882309F09AC08091BE06843011F01092C7
:104FC000810480912507882309F46FC080918004B3
:104FD000813009F07DCF1092800480916E04882387
:104FE00009F076CF0E947829882309F471CF1F91A8
:104FF0000F91EF9008950E94332A882309F0D9C0B9
:105000008091A805882309F4F9C083E00E94E31386
:10501000882379F081E080936E0480916E04882368
:1050200009F432C183E20E94051610929505109290
:10503000940580E00E94E313882309F0ECC01091EE
:10504000A805113009F4FFC080E00E94BA1388233C
:1050500009F089C09091A5058091E304981711F09B
:105060000E94E21F8091BE06813011F010928104EF
:1050700080912507882309F4B5CF84E00E942D2A6A
:105080000E947829882309F423CFB1CF0E94B41657
:1050900011E01093730484E20E9405168091BF060C
:1050A0000E94CB171093810441CF81E00E942D2AEA
:1050B00010926E048BCF81E08093990580E00E946E
:1050C000211680E00E94E313882309F46ECF11E0DB
:1050D0001093A80582E20E943D161093460480E0DA
:1050E0000E94BA13882309F466CF82E20E94051653
:1050F0001092A80580914604813009F4E6C0109210
:10510000460459CF0E94382C9091A505969590930E
:10511000ED04882309F033CF0E949D3230CF0E94E6
:10512000B41682E20E94051681E08093810481E238
:105130000E9405168091340660913A064091AD05B3
:1051400020913B0600913406E090AB050E940319C4
:1051500080916E04882309F49BC083E20E9421168B
:105160000E94141807CF82E20E9405161092A8052B
:105170002091A3053091A4052115310591F0E0910E
:10518000A505F0E0EE0FFF1FEB52FC4F80819181EF
:105190008217930730F021503040309395052093CB
:1051A000940580914604813009F480C01092460431
:1051B00051CF0E94B41682E20E940516109381041A
:1051C00081E20E943D168091340660913A0640913A
:1051D000AD0520913B0600913406E090AB050E949E
:1051E000031980916E04882309F456C083E20E945B
:1051F00005168091A805882309F007CF0E94382C56
:105200009091A50596959093ED04882309F0FDCE25
:105210000E949D32FACE11E01093A8051092A405C9
:105220001092A30582E20E943D1680919405909110
:10523000950501960E940302109346041091A8055B
:10524000113009F001CF0E940115482F882309F47D
:10525000FBCE41502091A3053091A405C901880FD0
:10526000991F880F991F880F991F220F331F820FD4
:10527000931F840F911D9093A4058093A3050E9412
:10528000030210934604E0CE83E20E943D16CDCE89
:1052900083E20E943D1664CF83E20E943D16B0CEA9
:1052A0008093980583E20E94051673CE80913406A0
:1052B00060913A064091AD0520913B06009134067D
:1052C000E090AB050E94031971CF80913406609184
:1052D0003A064091AD0520913B0600913406E090DE
:1052E000AB050E9403190BCF81E00E942D2ADECD71
:1052F0009091E2048091E804891731F08091E204F2
:105300008093E80481E0089580E0089580913B0651
:10531000882391F08091F3058093D7068091AB05A7
:10532000809318078091AD058093340680913B06E9
:1053300080933A0610923B0680913A06882329F022
:1053400080913A0680933A06089581E080933A0668
:1053500008958091F3058093D7068091AB058093E3
:1053600018078091AD058093340680913B068093A9
:105370003A0610923B060895833059F0843050F07D
:10538000843029F08091BF068093C606089510925C
:10539000BF0608958230B0F70895FC0187858F70AD
:1053A0008D30C1F030E020E190E080818F708E3050
:1053B00061F09F5F31969217C0F3892F913118F4F5
:1053C0008150832B089580E1FBCF9923B1F780E0D2
:1053D000832B089530E12FE0E7CF1F93DF93CF9326
:1053E0000F92CDB7DEB7162F0E94CD298983898110
:1053F0008F708F5F8093F7031093B105898184FDCF
:1054000008C08CE08093F5030F90CF91DF911F913E
:10541000089580E18093F5030F90CF91DF911F9164
:105420000895E82FF0E0EF73F070E750FC4F8081B3
:1054300008954093AF056093F2058093BE0681E026
:10544000809337060895882339F08091F205809380
:10545000BE0681E08093370608958093BE0681E002
:1054600080933706089580913706882319F01092AB
:10547000370681E008953F924F925F926F927F923C
:105480008F929F92AF92BF92CF92DF92EF92FF9254
:105490000F931F93CF93DF93462E4A015901662342
:1054A00009F4C4C09C01E90100E0FF241FEFDD24E2
:1054B00066247724B2E05B2E33243394CE010E941D
:1054C000CD29F301EE53F94F8083C0802FE0C22233
:1054D000C39440E050E012C01E251F7BF1F4F5019B
:1054E000E00FF11D3082FF2009F070C0DD24D3945D
:1054F0000F5F4F5F5F4F1E2D4C1588F5642FFE0127
:10550000E40FF51FE0802E2D30E0C9018F70907000
:105510000F9709F455C0DD20F9F6F501E00FF11DF4
:105520005082EF2DF0E0D401AE0FBF1FEC926295D8
:10553000607FE45CF94F6083F3940024220F331FF3
:10554000001C220F331F001C232F302DDD24D39489
:10555000D2220F5F4F5F5F4F1E2D4C1578F20894DB
:10556000611C711C6096641408F4A8CF003408F024
:1055700061C08F2DF501E00FF11D10820F5F003427
:10558000C8F39FE39F1550F09FEFEF2DF0E0E45C30
:10559000F94F9083F3942FE32F15B8F7DF91CF9154
:1055A0001F910F91FF90EF90DF90CF90BF90AF9041
:1055B0009F908F907F906F905F904F903F90089555
:1055C000F501E00FF11D1082DD2492CFEF2DF0E008
:1055D0003197E80DF91DE082FA94EF2DF0E0F39495
:1055E000E45CF94FA081AF70BA2FBF5F80818295D4
:1055F0008F70682F70E0CB018B0F911D40970CF0DE
:10560000BA2F0024220F331F001C220F331F001C4F
:10561000232F302DDD24D394D22262957295707F92
:105620007627607F7627B62BB08362CF00E0FF2419
:1056300080E0A0CF8F2DA5CF2F923F924F925F9207
:105640006F927F928F929F92AF92BF92CF92DF9292
:10565000EF92FF920F931F93CF93DF935C01562E2F
:105660003A016901662309F45DC0482EEC0130E07F
:1056700060E0EE24FF24FA9480E000E010E05FE0B8
:105680004EE0342E2DE0222E92EC892E96E0992EBB
:10569000800E911EF40170817F707F5FDE0190E0CB
:1056A000442D41950BC05C93223089F0E42EEA0E24
:1056B0003F5F9F5F1196822F9717D0F4F601E30F9B
:1056C000F11D2081213079F7882349F45C93F3019F
:1056D000E60FF11DF0806F5FFC9222E0E7CF5C9354
:1056E000F501EE0DF11D808180648083FC92DECF98
:1056F000903158F4FE01E90FF11D30829F5F05C023
:10570000FE01E90FF11D50839F5F9031C8F3F40152
:10571000808184FD2F860F5F1F4F6096822F0515B5
:1057200008F4B2CFDF91CF911F910F91FF90EF90CE
:10573000DF90CF90BF90AF909F908F907F906F90B1
:105740005F904F903F902F9008958091AF050E94F9
:10575000BA13882339F08091F2058093BE0681E068
:1057600080933706089510929E0584E20E943D16AC
:105770001092700480E00E943D160E944B180E9417
:105780004F170E94C9168091EC040E94D71680E042
:105790000E94951D089581E080939E0584E20E94F9
:1057A00005160E94C91680E00E94D71680E00E946C
:1057B000951D0895109239060E944F170E94C91630
:1057C0000E944B188091EC040E94D7161092350667
:1057D00081E20E943D1680E00E94951D10922507EF
:1057E0008CEF0E94F40F08951092AE0581E0809333
:1057F000350681E20E94051680E00E94951D809189
:105800003C04882321F480913D0480FDFCCF10925C
:105810003D04109254041092950480919504809355
:10582000970481E080933906809325078AEF0E94D0
:10583000F40F089580918104882311F480E0089585
:1058400081E00E94E313882321F081E080938204A9
:10585000089581E00E94A413882381F380E00E94D0
:105860008E13882359F382E08093820481E00895A7
:1058700088E00E948E13882369F09091BE0688E02C
:105880008093AF059093F20583E08093BE0681E09C
:1058900080933706089580913C04823011F080E0B7
:1058A00008950E94231080931A0780E00895AF9214
:1058B000BF92CF92DF92EF92FF920F931F93CF93FD
:1058C000DF935B01C82EDD24C294D29450EFD52221
:1058D000DC24C522DC24EE24C0E0D0E0FF24F394D5
:1058E00005C02196F394F1E1FF16B1F085010C0F8C
:1058F0001D1FC6018C0F9D1F0E94A41EF8018083EE
:10590000EE2079F780818F708E3059F7EF2C219639
:10591000F394F1E1FF1651F7EE20A1F490E1F501C7
:1059200087858F708D30B9F0892F81508F70DF910E
:10593000CF911F910F91FF90EF90DF90CF90BF908C
:10594000AF9008959E2D915051F791E0F501878514
:105950008F708D3049F7903110F08EE1E8CF892FAC
:1059600081508F708061E3CFBF92CF92DF92EF9230
:10597000FF920F931F93CF93DF936801E82EFF24CC
:10598000EE0CFF1CE60EF11CEE0CFF1CEE0CFF1CD7
:10599000EE0CFF1CE40EF11CE294F29470EFF7227F
:1059A000FE24E722FE2430E022953295307F322714
:1059B000207F3227B22E222379F0C0E0D0E086018A
:1059C0000C0F1D1FC7018C0F9D1F0E94A41EF80104
:1059D00080832196CB1598F3DF91CF911F910F9182
:1059E000FF90EF90DF90CF90BF900895EF92FF92DD
:1059F0000F931F93CF93DF93182F062F0E94141835
:105A0000E12EFF24EE0CFF1CEE0CFF1CEE0CFF1C25
:105A1000E00EF11CE294F294A0EFFA22FE24EA22B6
:105A2000FE24C0E0D0E0FE01E953F94F8081BE01C1
:105A30006E0D7F1D0E94601E2196C031D10599F721
:105A40000E941418DF91CF911F910F91FF90EF905A
:105A50000895CF92DF92EF92FF920F931F93CF930F
:105A6000DF93E22E6801082F10E0000F111F060FD0
:105A7000111D000F111F000F111F000F111F040F28
:105A8000111D02951295107F1027007F1027FF240B
:105A9000E294F29480EFF822FE24E822FE24FE2C09
:105AA00082E00E9405160E941418EE2089F0C0E0E2
:105AB000D0E0F601EC0FFD1F8081B8016C0F7D1F57
:105AC0000E94601E84E00E94E90E2196CF1588F3A3
:105AD00082E00E943D160E941418DF91CF911F9121
:105AE0000F91FF90EF90DF90CF900895EF92FF928B
:105AF0000F931F93CF93DF93182F062F0E94141834
:105B0000E12EFF24EE0CFF1CEE0CFF1CEE0CFF1C24
:105B1000E00EF11CE294F29440EFF422FE24E42221
:105B2000FE24C0E0D0E0CE018E0D9F1D0E94A41E79
:105B3000FE01E953F94F80832196C031D10599F7D1
:105B40001092700480E00E945A160E941418DF918F
:105B5000CF911F910F91FF90EF90089580913C0499
:105B6000882349F40E94A50080913C04813049F0CB
:105B70000E94391308950E94A60080913C04813050
:105B8000B9F70E94401308950F931F938091BF06A9
:105B90008093C60680913B068823C9F08091F30567
:105BA0008093D7068091AB05809318078091AD054F
:105BB0008093340680913B0680933A0610923B0610
:105BC00080917304823088F01F910F910895909115
:105BD00018078091AB059817B9F380917304823050
:105BE00098F78091AB05809318078091D706609154
:105BF00018074091340620913A060EE716E00E94FD
:105C0000B42C609134068091C0069091C1060E9428
:105C1000ED291F910F9108951092250780E00E94B1
:105C2000951D8CEF0E94F40F80913C04813011F09F
:105C30000E940F1310927C06109295048091950497
:105C4000809397041092AC058EE796E09093C1067E
:105C50008093C0068091E8048D3031F0833021F0CC
:105C60008B3011F0873011F40E94C42D80914A04CA
:105C7000882361F480914904882309F40895809170
:105C800049040E94CE0F10924904089580914A045D
:105C90000E94CE0F10924A04EDCF5F926F927F92D6
:105CA0008F929F92AF92BF92CF92DF92EF92FF922C
:105CB0000F931F93CF93DF9381E08093BE06809371
:105CC000370610E0C0E0D0E0BB24FF24F39432E0BC
:105CD000E32E20E1A22E9FE0992E84E0882E06E09C
:105CE000702EB7E06B2EA0E25A2E0E9453150E9430
:105CF0004E0C8091BE06863009F472C0873008F0E1
:105D0000ADC0813009F4E0C1843079F78091370665
:105D1000882339F010923706F092760410927404BA
:105D200010E08091AF050E94BA13882331F1809171
:105D3000F2058093BE06F09237061123E1F08091C0
:105D40007404882311F4F0927404809174048132F5
:105D500010F050927404909100028091740498178E
:105D600051F080917404809300026091000287E0FA
:105D700090E00E946802109246040E940115382F9C
:105D8000882389F0809174042AE0829FC001112445
:105D900080937404809174048150830F8093740401
:105DA000E092760411E080917604882309F49DCF77
:105DB0009091000280917604823009F4AFC2892F5D
:105DC00090E00E940302F0924604109276040E9432
:105DD00053150E944E0C8091BE06863009F08ECF7E
:105DE00080913706882339F0109237061092760496
:105DF0001092740410E08091AF050E94BA138823BA
:105E000049F08091F2058093BE06F0923706112387
:105E100009F087C280917404882309F411C220918B
:105E20007404213009F4EFC120917404223009F484
:105E3000BEC180917604813009F4DAC18091760484
:105E4000823009F052CF109276040E94C9168091D8
:105E5000AD040E94D7160E94141847CF8F3009F462
:105E6000E6C0803109F45FC0873009F03ECF8091F1
:105E70003706882321F010923706F092760480913D
:105E8000AF050E94BA13882351F08091F2058093E8
:105E9000BE06F09237068091760481FD4FC20E94C3
:105EA0008714882389F0982F9150933068F480915B
:105EB0003C04981749F090933C040E94AE2D8091C9
:105EC000760483608093760483E00E94A413882381
:105ED00079F0809179048F5F8093790480917904BF
:105EE0008170809379048091760483608093760436
:105EF0008091760480FFF9CE809176048E7F809326
:105F000076040E94BD1780913C048F5F0E945D174C
:105F100083E20E943D1680917904882309F422C20D
:105F20000E941418E2CE80913706882359F010920F
:105F30003706F09276041092F803F092740410E0A1
:105F4000C0E0D0E08091AF050E94BA138823B1F081
:105F50008091F2058093BE06F0923706112351F02E
:105F600080917404813009F440C2809174048230BD
:105F700009F408C210924604F092F80380E00E94EF
:105F8000A413882361F080917404823041F0E09280
:105F9000740482E20E942116F092760410E00E94BE
:105FA0000115282F882389F0CE01880F991F880FAB
:105FB000991F880F991FCC0FDD1FC80FD91F2150C3
:105FC000C20FD11DE092760411E0009174040230FA
:105FD00009F46AC180917604882309F486CE809101
:105FE0007404813009F478C180917404823009F01E
:105FF0007CCE80917604823009F025C20C2F8BE193
:106000000E943D168CE10E943D16002339F0B7FC3A
:1060100045C21B141CF48CE10E940516802F90E0F1
:106020000E940302F0924604109276045ECE8091A4
:106030003706882349F010923706F0927604809153
:10604000E3048093750410E08091AF050E94BA13B9
:10605000882349F08091F2058093BE06F0923706BE
:10606000112309F049C10E948714882369F0982FF1
:106070009150933048F48091A704981729F0909399
:10608000A704F092760411E08091A704813009F40E
:10609000EFC080917604882309F427CE109276040D
:1060A0000E94BD170E94C9168091A7048F5F0E94AD
:1060B0005D178091A704813009F017CE8091AA0462
:1060C00081500E94D71611CE80913706882331F077
:1060D000109237060E94B4160E94141887E10E949D
:1060E000E313882359F09091BE0687E18093AF05B2
:1060F0009093F2056092BE06F092370688E00E9407
:10610000E313882359F09091BE0688E08093AF0591
:106110009093F2057092BE06F092370681E00E94DD
:10612000E313882351F08091BE06F092AF0580936F
:10613000F2058092BE06F09237068EE00E94E313CD
:10614000882359F09091BE068EE08093AF0590931E
:10615000F2059092BE06F092370682E00E94E313A9
:10616000882351F08091BE06E092AF058093F2053E
:10617000A092BE06F09237069091E2048091E80466
:10618000891709F4B2CD8091E2048093E804DF918D
:10619000CF911F910F91FF90EF90DF90CF90BF9024
:1061A000AF909F908F907F906F905F9008959091A7
:1061B000E30480917504981759F08091E30480936B
:1061C000750420937604809175048093AD0411E0EA
:1061D00089E00E94BA13882309F42BCE109274042C
:1061E0008BE10E943D1680917604813009F026CE25
:1061F000109276040E94C9168091C0040E94D7169E
:106200000E94141872CD9091E30480917504981740
:1062100059F08091E3048093750420937604809173
:1062200075048093C00411E08AE00E94BA138823A9
:1062300009F4FACD109274048CE10E943D16F4CD5D
:106240008AE00E94A413882309F090C089E00E948C
:10625000A413882309F4E3CD8BE10E940516E09294
:106260007404E09276048091E30480937504D7CDA2
:10627000909175048091E304981709F40ACF8091F6
:10628000E30480937504909175049F5F923008F445
:10629000EAC08091AA04981709F4FBCE9093AA044F
:1062A000F092760411E0F5CE89E00E94A4138823D1
:1062B00031F01B1424F400937604BB24BA948AE0D2
:1062C0000E94A413882309F485CEB7FE83CEE09202
:1062D0007604BB24B3947ECE80917604823009F498
:1062E000C4C080918B0490918C040E940302F092B0
:1062F00046041092760478CE8091AA046091A70497
:1063000090E0019782959295907F9827807F9827BB
:10631000682B8AE090E00E946802A5CE90917404F8
:106320004ECD83E090E06091C0040E94680284E05A
:1063300090E06091AD040E9468026CCD8091790478
:1063400090E08170907082959295907F9827807FE1
:10635000982760913C046F70682B82E090E00E9467
:1063600068029DCD83E20E940516DACD8CE10E9481
:106370000516F0927404F09276048091E304809301
:10638000750464CFB7FC81C081E0C536D10508F043
:1063900073C0992787FD90958C9F60018D9FD00CCD
:1063A0009C9FD00C1124BC2C6C2D772767FD709519
:1063B000872F972F22EE34E040E050E00E941748EC
:1063C00060537D4E8C4E9F4F0C2DF89460930902C4
:1063D00070930A0280930B0290930C028DE090E080
:1063E000602F0E9468027894C5CDC431D10508F4AD
:1063F00040C081E0CD32D80710F0CCE2D1E0F89473
:1064000080918B0490918C048C179D07D1F0D093D0
:106410008C04C0938B0480918B0490918C040E9417
:10642000CC0280918B0490918C049093A40480936F
:10643000A30460918B0470918C0485E090E00E942D
:106440007202789492CD8DE090E00E946102282F34
:10645000992787FD909597FD1DC0082F27FD17C030
:10646000BB24B394CCCD92E014CFCE010E940302A2
:106470003ECFC4E1D0E0C3CFC0E0D0E0BB2460EDAC
:1064800072E183E190E000E0A0CF8FEF7ECFBB24EC
:10649000BA94B5CD909581959F4FDFCF8BE10E9447
:1064A0000516B7CD1F93DF93CF930F92CDB7DEB70D
:1064B00080E00E94951D10927C0610923D0410927F
:1064C0005404109283041092950480919504809353
:1064D00097041092AC058EE796E09093C1068093E6
:1064E000C006109134060E94CD29898389818F705E
:1064F0008F5F8093F7031093B105898184FD1BC0E2
:106500008CE08093F50383E0809325078AEF0E9457
:10651000F40F80913C04813011F00E94471383E016
:10652000809344041092490410924A040F90CF9132
:10653000DF911F91089580E1E4CFEF920F931F93B5
:10654000982F882309F495C0813029F080E01F91AD
:106550000F91EF90089580913706882309F0F9C0D4
:106560000E948714882399F1982F915080913B06BF
:10657000882341F4809134068093AD058091D7063D
:106580008093F3058091AD05891770F48091AD0576
:10659000981B9F5F90933B0680913B06853008F4E3
:1065A00046C184E080933B0680912507882309F447
:1065B00041C18091340660913A064091AD05209129
:1065C0003B060091B105E090AB050E94031984E100
:1065D0000E94A413882309F0DEC085E10E94A41361
:1065E000882309F0CEC080912507882321F590915A
:1065F00018078091AB059817F1F08091AB05809357
:1066000018078091D70660911807409134062091B1
:106610003A060EE716E00E94B42C80913406609191
:106620003A064091AD0520913B060091B105E090FE
:10663000AB050E94031980912507882329F48091D6
:106640003B06882309F0D4C00E94A114982F882308
:1066500009F47CCF809174049150981709F076CF9B
:106660008091F2058093BE0681E08093370680E03A
:106670006ECF0E948714982F8823D1F584E10E9461
:10668000A413882309F49FC01092AB0588E00E94F0
:10669000051681E00E943D1680912507882309F0A8
:1066A00055CF909118078091AB05981709F44ECFFC
:1066B0008091AB05809318078091D70660911807E9
:1066C0004091340620913A060EE716E00E94B42C61
:1066D0008091340660913A064091AD0520913B06C9
:1066E0000091B105E090AB050E94031980E02FCF27
:1066F0008091ED048093F30501E000933B06192F90
:1067000011501093AD0584E10E948E13882309F483
:106710004BC01092AB0588E00E94051681E00E94F4
:106720003D16109374048091BE068093F2058DE0AF
:106730008093BE0681E0809337061092BF06809159
:106740002507882309F44FC081E01F910F91EF9036
:1067500008951092370690938104809134066091D9
:106760003A064091AD0520913B060091B105E090BD
:10677000AB050E9403190E948714882309F427CFD0
:10678000F3CE81E08093AB0588E00E943D1681E066
:106790000E94051628CF1092AB0588E00E940516CE
:1067A00081E00E943D1619CF85E10E948E13882357
:1067B00009F4B7CF0093AB0588E00E943D1681E055
:1067C0000E940516AECF85E10E94A413882309F428
:1067D00063CF81E08093AB0588E00E943D1681E0A5
:1067E0000E94051659CF82E00E94BC2981E0ADCFFE
:1067F0008091F3058093D7068091AB0580931807AD
:106800008091AD058093340680913B0680933A06D3
:1068100010923B068091D70660911807409134068C
:1068200020913A060EE716E00E94B42C0DCF80911D
:106830003B06B8CE8091F3058093D7068091AB05D7
:10684000809318078091AD058093340680913B06B4
:1068500080933A0610923B068091D7066091180704
:106860004091340620913A060EE716E00E94B42CBF
:10687000A0CE2F923F924F925F926F927F928F9213
:106880009F92AF92BF92CF92DF92EF92FF920F93BF
:106890001F93DF93CF930F92CDB7DEB70E945315AE
:1068A0001092BF068091BF068093C606809125078F
:1068B000882311F40C94D13D84E08093BE0681E0DE
:1068C000809337066624992488245524772473946A
:1068D0003CE0432E23E0322E96E0292E0E945315F1
:1068E0000E944E0C1091BE061830E9F0193008F0E5
:1068F0004EC0153009F4A0C4163008F098C011300D
:1069000009F433C2143009F40EC40E944B2C8823BE
:1069100029F70E941A2C0E9453150E944E0C1091C8
:10692000BE06183019F780913706882349F0109277
:1069300037060E94B41683E20E9405167092730413
:106940008091AF050E94BA138823A1F08091F205CF
:106950008093BE0670923706109273048091D7061A
:10696000609118074091340620913A060EE716E030
:106970000E94B42C0E948714882309F00EC50E943F
:10698000A114882311F281500E94FB18BECF1B3046
:1069900009F4DEC21C30D0F5193009F485C21A3072
:1069A00009F0B3CF809137068823F9F010923706AB
:1069B00080E00E9405160E9414188091D70660910D
:1069C00018074091340620913A060EE716E00E941F
:1069D000292D80E00E943D160E94141884E08093C7
:1069E000BE06709237061092730480917604882355
:1069F00039F084E08093BE067092370610927604D8
:106A0000809176048F5F809376047FCF1C3009F4E9
:106A10007CC11D3009F079CF81E00E949D328091C8
:106A2000BE068D3009F471CF109281046ECF1630FE
:106A300009F4FCC0173009F068CF8091370688232D
:106A400089F1109237060E94B41660913A068EE7DB
:106A500096E048ED56E022EB35E00E943B2A80E0CC
:106A60000E9405161092760489E0809374041092B7
:106A7000750480913A06882391F020E0E22FF0E03F
:106A8000EE53F94F9081809175048F5F9F70890F4D
:106A9000809375042F5F80913A06281778F3662457
:106AA0009924552480E00E94E313882311F0662482
:106AB000639488E00E94E313882311F012E0612EB2
:106AC00087E10E94E313882311F0B3E06B2E8091DD
:106AD0007404893009F4E7C680917404813009F4A4
:106AE000BBC680917404882309F490C58091740416
:106AF000882329F080917404807F09F45FC010918D
:106B000074048EE00E94A413882351F080917404D1
:106B100080618093740485E080937604F2E05F2EB8
:106B20008FE00E94A413882351F080917404806246
:106B30008093740485E0809376045524539484E113
:106B40000E94A413882349F0809174048064809388
:106B5000740485E08093760455248EE00E94BA1375
:106B6000882341F080917404807E8093740484E0D3
:106B7000809376048FE00E94BA13882341F08091BD
:106B80007404807D8093740484E08093760484E1AF
:106B90000E94BA13882341F080917404807B809313
:106BA000740484E08093760480917604853009F43F
:106BB0004DC580917604843009F45FC580917404DA
:106BC000883009F43BC48091760490E08370907023
:106BD000892B09F04BC4662009F497CE60913A06E0
:106BE0008EE796E048ED56E022EB35E00E941C2B44
:106BF0008091D706609118074091340620913A069B
:106C00000EE716E00E94292D81E0681609F445C5BB
:106C100092E0691609F474C0E3E06E1609F075CECF
:106C2000F7E0F093BE06709237066FCE809137067C
:106C30008823D9F0109237060E94B41660913A0664
:106C40008EE796E048ED56E022EB35E00E943B2AC5
:106C500084E20E940516109276041092750493E661
:106C60009093740466249924882480E00E94E3139E
:106C7000882311F06624639488E00E94E31388233C
:106C800011F082E0682E80917404833609F41DC5EA
:106C900080917404813009F427C580917404833095
:106CA00009F485C580917404882309F450C4809147
:106CB000760490E083709070892B09F018C46620E8
:106CC00009F423CE60913A068EE796E048ED56E04F
:106CD00022EB35E00E941C2B8091D70660911807AB
:106CE0004091340620913A060EE716E00E94292DC5
:106CF00081E0681609F4D1C492E0691609F005CE66
:106D00002092BE067092370600CE80913706882307
:106D100089F0109237069091710480913A06981785
:106D200009F42CC6709276048091F2058093BE0619
:106D3000709237068091AF050E94BA13882309F438
:106D4000E4CD8091F2058093BE0670923706809163
:106D50007604882309F4B7C58DE00E943D1682E0D1
:106D60000E943D160E941418D0CD809137068823CA
:106D7000E9F01092370680E00E943F020E94B416AC
:106D800082E20E9405161093810481E20E943D1662
:106D90008091340660913A064091AD0520913B0602
:106DA00000913406E090AB050E94031980E00E9438
:106DB0009D3280E00E94A413882329F085E080930F
:106DC000BE067092370683E00E94A413882359F010
:106DD0008091BE063092AF058093F20588E08093E3
:106DE000BE067092370688E00E94E313882321F0E4
:106DF0002092BE067092370687E10E94E313882333
:106E000029F087E08093BE06709237068BE00E94DF
:106E1000E313882359F09091BE068BE08093AF0571
:106E20009093F2058093BE06709237068DE00E9423
:106E3000E313882359F09091BE068DE08093AF054F
:106E40009093F2054092BE06709237068091BE067E
:106E5000813011F01092810480912507882329F058
:106E600084E08093BE06709237069091E204809190
:106E7000E804891709F449CD8091E2048093E8047D
:106E80000F90CF91DF911F910F91FF90EF90DF90C6
:106E9000CF90BF90AF909F908F907F906F905F90BA
:106EA0004F903F902F90089580913706882371F07E
:106EB0001092370682E20E943D1681E00E94951DE5
:106EC00080E00E94951D80E00E943F029091740432
:106ED0008091B0059817C9F0909074048091B00526
:106EE0008093740480917604833009F4AAC580915C
:106EF0007604823050F08091AA05882331F4E09125
:106F00007404F0E0EE54FA4F708286E10E94A413FC
:106F1000882329F08091AA05882309F450C580911F
:106F20007604833009F4BEC386E10E94BA13882335
:106F300009F4EBCC80917604823009F0E6CC7092B3
:106F4000760480E00E94951D82E00E943D16DDCC13
:106F500080913706882361F01092370682E20E9402
:106F60003D168FE00E9405160E94141810927604B8
:106F70008091AF050E94BA13882309F442C0809122
:106F8000F2058093BE0670923706809176048823BE
:106F900091F58091D706309118072091340690E042
:106FA000880F991F830F911D880F991F880F991FB4
:106FB000880F991F280F2093720480913A068093BE
:106FC00071048823C1F090E0A0E0B0E0282F30E009
:106FD00022953295307F3227207F3227FD01E258FB
:106FE000F94F8081AC50BA4F8C939F5FA92FB0E0CE
:106FF000A217B3079CF38FE00E943D168DE00E941C
:107000003D168DE00E94A413882309F47ECC809164
:107010007604882309F079CC80917104882309F4DF
:1070200074CC709276048091D70620911807109145
:10703000340690E0880F991F820F911D880F991FC9
:10704000880F991F880F991F180F809172041817C5
:1070500009F45BCC8DE00E94051682E00E940516C3
:107060000E9414186091720480913A06882309F4F2
:1070700040C0C62EDD24C294D294A0EFDA22DC24D4
:10708000CA22DC24A12EBB24A294B294F0EFBF222A
:10709000BA24AF22BA24750100E010E0C6010E94B4
:1070A000A41E882E0258194FF8018083C7010E9440
:1070B000A41EB6010E94601E882DB7010E94601EAA
:1070C00084E00E94E90E0894C11CD11C0894E11CC4
:1070D000F11C8E2D8A19082F10E080913A0690E05D
:1070E00082959295907F9827807F98270817190797
:1070F000ACF2109134068EE796E00E94CD29898388
:1071000089818F708F5F8093F7031093B105898118
:1071100084FD51C58CE08093F50382E00E943D160A
:107120000E941418F2CB809137068823E9F0109260
:1071300037060E94B41682E20E94051670928104FE
:1071400081E20E9405168091340660913A064091D2
:10715000AD0520913B0600913406E090AB050E94FE
:10716000031981E00E943F0283E00E94E313882319
:1071700009F445C080913B06882309F00DC4909125
:1071800018078091AB05981781F08091AB0580932B
:1071900018078091D7066091180740913406209116
:1071A0003A060EE716E00E94B42C60913A068EE78C
:1071B00096E048ED56E022EB35E00E943B2A80E065
:1071C00090E0FC01EE54FA4F108201968034910554
:1071D000C1F782E08093730410921B07109275042C
:1071E00010927404109276041092AA05709278049A
:1071F00089E08093BE067092370699249A94809114
:10720000BE06843011F010928104809125078823F6
:1072100021F47092BE06709237068091800481300E
:1072200009F073CB109280049091E2048091E804FD
:10723000891709F021CE69CB809137068823C9F0E0
:10724000109237060E94B416709276048EE796E08C
:107250000E94CD29282F2F702F5F2093740490E077
:10726000929582958F7089279F708927817080936E
:1072700075048EE00E942215823009F4D2C08AE0A3
:107280000E942215823009F4C3C089E00E942215B1
:10729000823009F4B1C08FE00E94A413882391F0DA
:1072A0003092760480917504882311F4409274041E
:1072B000809175048F5F809375048091750481704F
:1072C000809375048091760480FF21C080917604BC
:1072D00081508093760480917504882309F4AAC1B3
:1072E00080917404803108F4A9C381E08093740410
:1072F00083E00E94051680917404882309F097C1E9
:1073000081E080937404809174040E94ED1680E003
:107310000E94BA13882309F4F8CA80917604823057
:10732000B8F182E0809373048EE796E061E048ED67
:1073300056E022EB35E00E943B2A90917404809144
:107340007504811180E191509F70892B8093C20652
:107350008EE796E061E048ED56E022EB35E00E94D2
:107360001C2B8091D706609118074091340621E0CC
:107370000EE716E00E94292D8091D706609118072C
:107380004091340620913A060E94B42C1092730466
:107390007092BE0670923706B8CA182F1150812F0E
:1073A0000E94F3188091D70690911807E82EFF24C9
:1073B000EE0CFF1CE90EF11CEE0CFF1CEE0CFF1C8A
:1073C000EE0CFF1CE10EF11CE294F29450EFF5225A
:1073D000FE24E522FE248701005F1F4F8FE0B701E6
:1073E0000E94601E84E00E94E90E0894E11CF11CDA
:1073F000E016F10699F7C3CA8091740490E00E96E6
:107400008F7090708F5F809374043092760443CFB6
:10741000809174048F708F5F80937404309276042F
:1074200034CF80917604823008F483C38091740451
:107430008F5F809374043092760421CFE92DF0E0C1
:10744000EE54FA4F5082939480917504981610F080
:10745000662463947092760410927404809176048A
:1074600090E083709070892B09F4B5CB0E94C91607
:1074700080913A068823B1F090E080E001C08E2F21
:10748000E92FF0E0EE53F94FE081EF70EF5FE80F86
:10749000981618F09E1608F4DDC29F5F80913A0698
:1074A000981768F384E00E943D1683E00E943D1621
:1074B00088E00E943D168091760480FD13C0E2E0D2
:1074C0005E1609F47AC3F1E05F1609F47AC3552019
:1074D00031F084E00E94051683E00E94051688E0E2
:1074E0000E9405160E9414181092760474CB0E9414
:1074F000C916E92DF0E0E45CF94F80818F3FD1F0AF
:10750000108112951F7000810F70010F0F5F10170F
:1075100038F010C0812F0E940B171F5F101750F416
:107520008091760480FDF6CF812F0E94D7161F5FD1
:107530001017B0F38091760480FFC0C1882D60E001
:107540000E945E19109276040E941418B8CB86E14E
:107550000E94A413882309F0B9C20E943914882319
:1075600009F082C287E10E94BA13882329F0FFE361
:107570009F0E9F22709276048EE00E94A4138823AF
:1075800021F080E1882A709276048FE00E94A41393
:10759000882321F090E2892A7092760484E10E9487
:1075A000A413882321F0E0E88E2A7092760485E106
:1075B0000E94A413882321F0F0E48F2A70927604AD
:1075C0008EE00E94BA13882321F08FEE88227092F9
:1075D00076048FE00E94BA13882321F09FED892260
:1075E0007092760484E10E94BA13882321F0EFE7B9
:1075F0008E227092760485E10E94BA13882309F4E2
:1076000056CBFFEB8F227092760451CB86E10E941D
:10761000E313882309F46ACAE92DF0E0EE54FA4F27
:1076200050807092740482E0809376045FCA8091E7
:10763000740467CE80917404813108F4FCC181E048
:107640008093740483E00E943D1655CE112309F007
:10765000E9C180917404882309F4E4C1662029F407
:10766000E92DF0E0EE54FA4F508282E080937604E8
:1076700080917604843009F0A1CA112359F08091D9
:107680007404882339F4939480917504981610F04B
:10769000662463947092760491CA6092BE066092EA
:1076A000370633C90E94D114882309F43DCC82E007
:1076B0008093760486E10E948E13882309F034CCEF
:1076C000709276040E94951D2FCC88E00E94BA1318
:1076D000882309F4DDCA10927404709276048091B4
:1076E0007404813009F0D9CA86E10E94BA13882354
:1076F00009F024C28EE00E94A413882349F0882D4B
:1077000080958071EFEE8E22882A82E08093760445
:107710008FE00E94A413882349F0882D8095807201
:10772000FFED8F22882A82E08093760484E10E9414
:10773000A413882349F0882D809580789FE78922BB
:10774000882A82E08093760485E10E94A41388232E
:1077500049F0882D80958074EFEB8E22882A82E094
:10776000809376040E943914182F882309F495CA4F
:1077700080E00E94951D85E00E94E90E11501F7067
:10778000F0EF8F22812AE82DF0E0EF73F070E750E0
:10779000FC4F482D4078808160E00E947E1D82E091
:1077A0008093760480917404833009F07BCA0E9430
:1077B0003914182F0E945314882319F4112309F443
:1077C00071CAE92DF0E0E852F94F808280E00E9412
:1077D000951D85E00E94E90E93948FE3891518F4B6
:1077E00010927504992470927604109274041123F7
:1077F00009F458CA812E8A949FE089228EE00E9463
:107800008E13882311F0E0E18E2A8FE00E948E1300
:10781000882311F0F0E28F2A84E10E948E138823DE
:1078200011F080E8882A85E10E948E13882311F0E8
:1078300090E4892AE82DF0E0EF73F070E750FC4FF8
:10784000482D4078808160E00E947E1D82E0809318
:1078500076043092740426CA86E10E94BA13882303
:1078600019F088E0809374048EE00E94A4138823AA
:1078700029F082E080937604A2E05A2E8FE00E94E5
:10788000A413882329F082E080937604552453942E
:1078900084E10E94A413882309F423C982E0809321
:1078A000760455241EC987E10E94BA13882309F47F
:1078B00013C910927404709276040EC9882D61E089
:1078C0000E945E193FCE82E00E9405160E941418A5
:1078D0009091D70620911807309134068091710459
:1078E0008823B9F1E92EFF24EE0CFF1CE20EF11CF7
:1078F000EE0CFF1CEE0CFF1CEE0CFF1CE30EF11C4B
:10790000E294F29450EFF522FE24E522FE24870152
:10791000A0E0B0E0FD01EC50FA4F8081A258B94FD1
:107920008C93B8010E94601E84E00E94E90E0F5FF4
:107930001F4F802F8E19A82FB0E08091710490E026
:1079400082959295907F9827807F9827A817B907EE
:107950000CF3109134068EE796E00E94CD298983BE
:1079600089818F708F5F8093F7031093B1058981B0
:1079700084FDE2C08CE08093F503EEC9992309F4FD
:10798000D1C982E20E943D168DE00E9405160E9438
:10799000141810927604CEC98091F3058093D7060F
:1079A0008091AB05809318078091AD0580933406D4
:1079B00080913B0680933A0610923B06EACB82E028
:1079C000809376040E94BB14882311F030927604D1
:1079D000E0917404F0E0EE54FA4F82E08083E0918D
:1079E0007504F0E0E852F94F808080923806E82D67
:1079F000F0E0EF73F070E750FC4F482D4078808145
:107A000060E00E947E1D80917404981639F0909079
:107A10007404809175048F5F8093750482E00E94E6
:107A200005167DCA939480917504981608F416CEB5
:107A3000662463941ACE8091740402CE80917404FB
:107A400055CC0E94BB14882309F051CA82E0809370
:107A500076044DCA992D981B8091760480FF9DC0B5
:107A6000892F0E940B171ECD882E8A94EFE08E225C
:107A70008EE00E948E13882311F0F0E18F2A8FE0B0
:107A80000E948E13882311F080E2882A84E10E94EC
:107A90008E13882311F090E8892A85E10E948E13C5
:107AA000882311F0E0E48E2AE82DF0E0EF73F07007
:107AB000E750FC4F482D4078808160E00E947E1D99
:107AC00082E080937604309274044CCDE92DF0E08E
:107AD000E852F94F80808EE00E948E13882311F0C7
:107AE000E0E18E2A8FE00E948E13882311F0F0E2ED
:107AF0008F2A84E10E948E13882311F080E8882A5F
:107B000085E10E948E13882311F090E4892AE82DE4
:107B1000F0E0EF73F070E750FC4F482D4078808123
:107B200060E00E947E1D82E080937604709274046F
:107B300014CD109274047ACC80E11DCFE92DF0E0D1
:107B4000E852F94F80828EE00E948E13882381F5DF
:107B500088248FE00E948E13882311F0E0E28E2AA1
:107B600084E10E948E13882311F0F0E88F2A85E1CA
:107B70000E948E13882311F080E4882A80E00E94FE
:107B8000951D93949FE3991518F410927504992408
:107B90007092760410927404ADCD892F0E94D7168E
:107BA00081CC81E08093BE06809337060C946234CA
:107BB00000E1802ECECF80E1AECA84E00E9405169F
:107BC00091CC83E00E9405168DCC0F931F93CF9329
:107BD000DF93EC01442319F18B0150E070E020E0C9
:107BE00030E0F901EE53F94F60816F706F5FD8019B
:107BF00090E0FE01E50FF11D80818D939F5F5F5F37
:107C00009617B8F3760F2F5F3F4F005F1F4F241773
:107C100040F3872FDF91CF911F910F91089570E06E
:107C2000872FDF91CF911F910F910895BF92CF922F
:107C3000DF92EF92FF920F931F93CF93DF936B012D
:107C4000B42E442369F17C0110E000E0C0E0D0E0F4
:107C5000C7010E94CD29FE01EE53F94F8083208198
:107C60002F702F5FD70190E08D91F601E10FF11D8C
:107C700080839F5F1F5F9217B8F3020F219680E108
:107C800090E0E80EF91ECB1518F3802FDF91CF910D
:107C90001F910F91FF90EF90DF90CF90BF900895CC
:107CA00000E0F3CFCF92DF92EF92FF920F931F93FA
:107CB000DF93CF93CDB7DEB7C054D0400FB6F89462
:107CC000DEBF0FBECDBF109276041092740482E026
:107CD0008093730440913A068EE796E06E01089413
:107CE000C11CD11CB6010E94163EE82E809175047D
:107CF0008E1510F01092750480913A068823C1F019
:107D000090E030E0E32FF0E0EE53F94F20812F7048
:107D10002F5F80E0E92FF0E0E45CF94F80838F5F14
:107D20009F5F8217B8F33F5F80913A06381750F390
:107D30000E94531580912507882309F4C9C184E066
:107D40000E942D2AFF240E9453150E944E0C109170
:107D5000BE06113081F01430F1F10E944B2C8823C3
:107D600091F70E941A2C0E9453150E944E0C1091FC
:107D7000BE06113081F70E94332A882309F0F4C02F
:107D800086E10E94E313882329F0809177048823F9
:107D900009F088C18091BE06813011F010928104F3
:107DA00080912507882309F070C10E9478298823D3
:107DB000A1F210927304C05CDF4F0FB6F894DEBFDF
:107DC0000FBECDBFCF91DF911F910F91FF90EF902C
:107DD000DF90CF9008950E94332A882309F037C19D
:107DE00010E086E10E94E313882309F0D0C087E108
:107DF0000E94E313882309F0E6C086E10E94BA13CB
:107E0000882309F0FCC087E10E94BA13882309F097
:107E100001C186E10E94A413882309F006C18EE007
:107E20000E94A413882339F08F2D809580719FEED6
:107E3000F922F82A12E08FE00E94A413882339F077
:107E40008F2D809580729FEDF922F82A12E084E14F
:107E50000E94A413882339F08F2D809580789FE7A6
:107E6000F922F82A12E085E10E94A413882339F050
:107E70008F2D809580749FEBF922F82A12E00E94E2
:107E80003914282F882361F08F2D90E08F70907027
:107E90000D9734F421502F7080EFF822F22A12E06F
:107EA00088E00E94A413882309F44AC08F2D90E033
:107EB0008F7090700D970CF4ECC090EFF92200E0F9
:107EC00010E080917504F601E80FF11DF0824091F9
:107ED0003A06C6016EE776E00E94E53DE82E81E0B5
:107EE000809377040D301105BCF58F2D61E00E9461
:107EF0005E1984E20E9405160E94C916E09175047D
:107F0000F0E0E45CF94F80810E94D7160E941418BB
:107F10008091BE06843011F0109281048091250773
:107F2000882309F4AEC080918004813009F015CF18
:107F3000109280040E947829882309F40ECF39CF4B
:107F4000123009F4C9C0113019F70F2D10E00F706D
:107F500010700D3011054CF28F2D60E00E945E19FB
:107F600084E20E943D16C8CF0E94B41682E20E94AD
:107F700005161093810481E20E943D1680917704DA
:107F8000882309F4A1C082E00E942116F9CE8091D5
:107F900075048F5F80937504809175046E2D0E9427
:107FA00036489093750480917504F601E80FF11D31
:107FB000F08082E00E94051611E087E10E94E31341
:107FC000882309F41ACF809175046E2D70E090E03B
:107FD0000197860F971F0E945648809375048091E1
:107FE0007504F601E80FF11DF08080E00E9405168F
:107FF00011E086E10E94BA13882309F404CF82E0DD
:108000000E943D160E94141887E10E94BA1388232B
:1080100009F4FFCE80E00E943D160E94141886E10C
:108020000E94A413882309F4FACE80E00E948E13E4
:10803000882309F4F4CE8091B00580937504809173
:108040007504F601E80FF11DF08011E0E8CE0E9402
:10805000B41682E20E94051681E08093810481E2D9
:108060000E940516809177048823C1F082E00E9467
:10807000211680917504F601E80FF11DF08011E0E2
:10808000B0CE81E00E942D2A4ECF84E00E942D2A9E
:108090008CCE8FE0F82E0FE010E013CF82E00E942C
:1080A0003D16E7CF82E00E943D168091D706609191
:1080B00018074091340620913A060EE716E00E9418
:1080C000292D1092770466CE82E00E943D1658CE8C
:1080D00081E00E942D2A36CE0F2D10E00F70107017
:1080E000F0CE3F924F925F926F927F928F929F92CB
:1080F000AF92BF92CF92DF92EF92FF920F931F93B6
:10810000DF93CF93CDB7DEB7C058D0400FB6F89409
:10811000DEBF0FBECDBF109276041092740482E0D1
:108120008093730440913A06B1E4CB2ED12CCC0E4F
:10813000DD1E8EE796E0B6010E94163EF82E0E94E4
:10814000531580912507882309F430C684E00E94E6
:108150002D2A9924442488245524AA24AA94BB2493
:10816000332433943E010894611C711C0E94531502
:108170000E944E0C1091BE061F30B9F0103108F06D
:108180008AC0113009F4BAC2143009F44EC20E94F8
:108190004B2C882359F70E941A2C0E9453150E94D9
:1081A0004E0C1091BE061F3049F70E94332A8823D7
:1081B00009F09BC40E94A52B86E10E94A41388238A
:1081C00009F08AC489E00E94A413882309F0D5C26B
:1081D0008AE00E94A413882309F0C7C286E10E94A6
:1081E000BA13882309F0BDC289E00E94BA1388231C
:1081F00009F0B3C28AE00E94BA13882309F0A9C229
:108200008DE00E94A413882329F0809171048823B3
:1082100009F031C591E0991609F4DBC3A2E09A1682
:1082200009F4D3C3B3E09B1609F0B1CF30927704C1
:10823000682D70E0842D992787FD9095860F971FF4
:10824000850D911D0E945648582EFF2099F020E080
:1082500030E0F601E20FF31F852D820F682D0E949A
:108260003648D301A90FB11D8C9180832F5F3F4FFA
:108270002F1578F340913A06C6016EE776E00E942A
:10828000E53D40913A068EE796E0B6010E94163E23
:10829000F82E99247CCF113109F41BC1113108F457
:1082A00080C0123109F073CF0E94332A882309F06D
:1082B00056C40E94A52B8CE00E94A413882309F0C9
:1082C00077C38CE00E94BA13882309F06DC38EE057
:1082D0000E94A413882309F05DC38FE00E94A413B9
:1082E000882309F04DC384E10E94A413882309F078
:1082F0003DC385E10E94A413882309F02DC388E0C3
:108300000E94A413882309F01DC38EE00E94BA13B3
:10831000882309F0EFC28FE00E94BA13882309F086
:10832000F2C284E10E94BA13882309F0F5C285E104
:108330000E94BA13882309F0F8C288E00E94BA1399
:10834000882309F0FBC2992009F421CF30927704E9
:10835000FF2009F48FCF860110C00E97F9F08E2D03
:108360008A21D8019C919B21892BF80181938F014F
:108370008E2F8C198F1508F07DCF0E94F800E82E03
:1083800090E08F7090708D30910539F7E7EFEE2215
:108390008E2D90E08F7090700E9709F7F7EFEF2217
:1083A000DECF0E94332A882309F09EC20E94A52BAB
:1083B0008CE00E94A413882309F0E7C187E10E94A2
:1083C000A413882309F0ECC180E00E94A413882341
:1083D00009F0F1C18CE00E94BA13882309F0F6C1BC
:1083E00087E10E94BA13882309F0F9C180E00E9456
:1083F000BA13882309F0FCC18EE00E94A4138823DD
:1084000009F0FFC18FE00E94A413882309F008C27D
:1084100084E10E94A413882309F011C285E10E941F
:10842000A413882309F01AC288E00E94A4138823A9
:1084300009F023C28EE00E94BA13882309F02CC2EF
:108440008FE00E94BA13882309F02FC284E10E94B2
:10845000BA13882309F032C285E10E94BA13882337
:1084600009F035C288E00E94BA13882309F038C2A7
:10847000992009F48CCE30927704E2E09E1609F43C
:10848000D0C3F4E09F1609F446C4B1E09B1609F08E
:1084900003C4FF2009F4EECE860107C00F5F1F4F13
:1084A000802F8C198F1508F0E5CE0E94F800E82E79
:1084B000EFE1E81798F30E94F800D8012C916F2D96
:1084C0000E943648F601E90FF11D80818C932083CC
:1084D000E5CF0E94332A882309F0F9C20E94A52B18
:1084E0008CE00E94A413882309F0E8C28CE00E946B
:1084F000BA13882309F0DEC28EE00E94A4138823F9
:1085000009F0CEC28FE00E94A413882309F0BEC2F6
:1085100084E10E94A413882309F0AEC285E10E9481
:10852000A413882309F09EC288E00E94A413882324
:1085300009F08EC28EE00E94BA13882309F084C22B
:108540008FE00E94BA13882309F05FC284E10E9481
:10855000BA13882309F062C285E10E94BA13882306
:1085600009F065C288E00E94BA13882309F068C246
:108570008DE00E94A413882329F080917104882340
:1085800009F043C0192D10FF02CE3092770411FD7F
:10859000EFC2FF2041F1860106C00F5F1F4F802F01
:1085A0008C198F1500F50E94F800E82EBFE3B8176C
:1085B000A0F30E94F800E82E90E08F7090708D304C
:1085C000910509F404C30E9709F4FEC29E2D9A2169
:1085D000D8018C918B21982B9C930F5F1F4F802F7C
:1085E0008C198F1500F3BEEF9B2240913A06C6010D
:1085F0006EE776E00E94E53D40913A068EE796E010
:10860000B6010E94163EF82EC2CD892D809582704B
:10861000B1E09B22982A8DE00E943D16192D91FC15
:10862000A2C388240E941418AECF0E94332A882344
:1086300009F07FC284E00E94E313882309F072C22C
:1086400085E00E94E313882309F065C282E10E945D
:10865000E313882309F058C281E10E94E3138823C1
:1086600009F04BC286E10E94E313882329F0809130
:108670007704882309F0EDC287E10E94E313882381
:1086800029F080917704882309F0B2C28091BE0658
:10869000843041F01092810482E00E943D1682E213
:1086A0000E943D1680912507882309F48AC1809194
:1086B0008004813009F06BCD109280040E947829EB
:1086C000882309F464CD10927304C058DF4F0FB6AD
:1086D000F894DEBF0FBECDBFCF91DF911F910F91F8
:1086E000FF90EF90DF90CF90BF90AF909F908F90D2
:1086F0007F906F905F904F903F9008950E94332A33
:10870000882389F48091BE06813011F01092810493
:1087100080912507882309F027C20E9478298823A1
:1087200009F435CDD0CF0E94B41682E20E9405161E
:108730001093810481E20E943D1680917704882382
:1087400009F4A6C282E00E94211681E00E943F0245
:10875000D9CF8CE10E943D1653CD8BE10E943D168E
:1087600049CD82E00E943D163FCD8CE10E94051666
:108770009E2C93944424439431CD8BE10E940516A2
:108780009E2C939444244A9423CD8EE00E94051697
:108790009924939487E10E94A413882309F414CEAA
:1087A00080E00E940516F2E09F2E80E00E94A41354
:1087B000882309F40FCE82E20E940516E3E09E2E84
:1087C0008CE00E94BA13882309F40ACE8EE00E943E
:1087D0003D1687E10E94BA13882309F407CE80E092
:1087E0000E943D1680E00E94BA13882309F404CE4B
:1087F00082E20E943D168EE00E94A413882309F4B1
:1088000001CE84E00E94051674E0972E60E1A62E4A
:108810005FEEB52E8FE00E94A413882309F4F8CDF3
:1088200083E00E94051644E0942E30E2A32E2FED43
:10883000B22E84E10E94A413882309F4EFCD88E0CE
:108840000E94051694E0992E80E8A82E0FE7B02E1E
:1088500085E10E94A413882309F4E6CD81E00E94FB
:10886000051614E0912EB0E4AB2EAFEBBA2E88E0E3
:108870000E94A413882309F4DDCD84E20E9405162A
:10888000F4E09F2EEFE0AE2E70EFB72E8EE00E9448
:10889000BA13882309F4D4CD84E00E943D168FE0FA
:1088A0000E94BA13882309F4D1CD83E00E943D16BB
:1088B00084E10E94BA13882309F4CECD88E00E9497
:1088C0003D1685E10E94BA13882309F4CBCD81E0DF
:1088D0000E943D1688E00E94BA13882309F4C8CD8F
:1088E00084E20E943D16C4CD89E10E9405169924B8
:1088F00044245CCD84E00E943D168FE00E94BA13B0
:10890000882309F40ECD83E00E943D1684E10E9485
:10891000BA13882309F40BCD88E00E943D1685E147
:108920000E94BA13882309F408CD81E00E943D1605
:1089300088E00E94BA13882309F405CD84E20E94DE
:108940003D1601CD84E20E940516992493942FE0F0
:10895000A22E90EFB92ED9CC81E00E940516992461
:10896000939440E4A42E3FEBB32EC9CC88E00E9440
:1089700005169924939460E8A62E5FE7B52EB9CC2E
:1089800083E00E94051699249394E0E2AE2E7FEDD9
:10899000B72EA9CC84E00E94051699249394A0E1F7
:1089A000AA2EFFEEBF2E99CC8EE00E943D168FCCF2
:1089B0008EE00E94051699249394AA24AA94BB24BD
:1089C00080CC81E00E942D2A72CE442009F02ECC6A
:1089D000DECB442009F4DBCB90927704FF2089F0B2
:1089E000342D3F0DD60120E0822F830F6F2D0E9482
:1089F0003648F301E90FF11D8D9180832F5F2F150C
:108A000098F340913A06C30138CC83E00E943D16AA
:108A100084E10E94BA13882309F49ECD88E00E9465
:108A20003D1685E10E94BA13882309F49BCD81E0AD
:108A30000E943D1688E00E94BA13882309F498CD5D
:108A400084E20E943D1694CD84E00E943D1678CDCC
:108A500084E20E940516A1E09A2A1FE0A12EB0EF41
:108A6000BB2E68CD81E00E94051691E0992A80E432
:108A7000A82E0FEBB02E58CD88E00E94051681E09D
:108A8000982A20E8A22E9FE7B92E48CD83E00E94C5
:108A90000516F1E09F2A40E2A42E3FEDB32E38CD1B
:108AA00084E00E940516E1E09E2A60E1A62E5FEEBA
:108AB000B52E28CD8EE00E943D161ECD8EE00E9480
:108AC0000516B1E09B2AAA24AA94BB240FCD8CE002
:108AD0000E940516992402CD82E00E94051640905E
:108AE000B0054194992493946DCB80E20E940516C1
:108AF00099244424EE2455245DCB6091BE0681E187
:108B000041E10E94192AAECD6091BE0682E142E1A8
:108B10000E94192AA1CD6091BE0680E145E00E9425
:108B2000192A94CD6091BE068FE044E00E94192A74
:108B300087CD0E94B41682E20E940516309281040D
:108B400081E20E94051680917704882309F47DC094
:108B500082E00E94211681E00E943F026BCD8BE0F3
:108B60000E9405169924A5CB84E00E942D2AD5CD1C
:108B7000FF2009F438CD860107C00F5F1F4F802FFB
:108B80008C198F1508F02FCD0E94F800E82EEFE326
:108B9000E81798F30E94F800682D0E943648F30108
:108BA000E90FF11DE0808E2D90E08F7090708D3078
:108BB0009105B9F00E9791F09E2D9A21D8018C91D4
:108BC0008B21982B9C93D9CFF7EFEF22FFCCE7EFC7
:108BD000EE228E2D90E08F709070F5CC87EFE8221A
:108BE000EBCFF7EFEF228E2D90E08F709070E2CFF9
:108BF00082E00E943D168091D7066091180740914F
:108C0000340620913A060EE716E00E94B42C4091FB
:108C10003A06C801B6010E94163EF82E109277045B
:108C200035CD8F2D869509F425CBD6016F2D61505A
:108C3000262F281B8C91F601E60FF11D90819D9344
:108C4000808361506217B1F715CB82E00E943D1618
:108C500082CF82E00E943D168091D706609118076E
:108C60004091340620913A060EE716E00E94292D25
:108C70001092770401CDE39481E0E8228DE00E9418
:108C80003D16EE2009F07BC088240E941418C2CA49
:108C900082E00E943D1659CD60913A068EE796E03B
:108CA000A60122EB35E00E943B2AF82E882311F121
:108CB000860106C00F5F1F4F802F8C198F15D0F4CF
:108CC0000E94F800E82EBFE3B817A0F30E94F80056
:108CD000F80120816F2D0E943648F601E90FF11D41
:108CE0008081D8018C9320830F5F1F4F802F8C19B8
:108CF0008F1530F360913A068EE796E0A60122EBDD
:108D000035E00E941C2B40913A068EE796E0B601B2
:108D10000E94163EAFCAFF2009F4ACCA860107C004
:108D20000F5F1F4F802F8C198F1508F0A3CA0E9468
:108D3000F800E82E8FE38E1598F30E94F800D80112
:108D40002C916F2D0E943648F601E90FF11D8081AC
:108D50008A219B2D9223892B8C9380818B212A2120
:108D6000822B8083DDCF8DE00E94051684EF95E095
:108D7000B301409171040E94163E882E53CC8DE0C1
:108D80000E94051684EF95E0B301409171040E94A2
:108D9000163E882E40913A068EE796E0B6010E9474
:108DA000163EF82EA3E09A2E44246FCF81E00E9455
:108DB0002D2ACFC9EF92FF920F931F930E94531554
:108DC00080912507882309F42EC184E00E942D2A72
:108DD000FF24F39407C0113009F478C00E944B2C93
:108DE0008823E1F00E9453150E944E0C1091BE069C
:108DF0001330F1F0143078F3143009F440C01D3012
:108E000069F781E00E949D328091BE068D3031F37A
:108E1000109281040E944B2C882321F70E941A2C67
:108E20000E9453150E944E0C1091BE06133011F78C
:108E30000E94332A882309F0B3C00E94A52B8823FF
:108E400021F010927304109281040E943914882337
:108E500009F093C080912507882309F0BFCF86E1F0
:108E60000E94A413882309F0D3C086E10E94BA139C
:108E7000882309F4B3CF80E00E94951DAFCF0E94F4
:108E8000332A882309F0A0C080E00E949D32882305
:108E900009F497C08091BE06843011F010928104CD
:108EA00080912507882309F4ABC08091800481302C
:108EB00009F094CF109280040E947829882309F445
:108EC0008DCF1F910F91FF90EF9008950E94332A4C
:108ED0008823B9F580E00E949D32182F86E10E9418
:108EE000A413882319F586E10E94BA138823D1F4CC
:108EF0001123A9F08091BE06813011F010928104F7
:108F000080912507882309F07FC00E947829882353
:108F100009F464CF1F910F91FF90EF9008950E9484
:108F2000382CE8CF80E00E94951DE2CF80E00E94BF
:108F3000112A9091C606890F60E040E00E947E1DD4
:108F4000D2CF0E94B41682E20E94051610938104CB
:108F500081E20E943D168091340660913A0640916C
:108F6000AD0520913B0600913406E090AB050E94D0
:108F7000031981E00E943F02ADCF182F11500E94CB
:108F8000F417812F0E94CB171093BF0680912507FD
:108F9000882309F05FCF8091BF068093C6065ACF21
:108FA0000E94B416F092730481E00E943F0284E2B2
:108FB0000E9405168091BF060E94CB17F092810493
:108FC0003CCF0E94382C66CF0E94B41682E20E94E9
:108FD0000516F092810481E20E9405168091340604
:108FE00060913A064091AD0520913B060091340610
:108FF000E090AB050E94031981E00E943F0244CF3C
:1090000081E00E942D2A51CF84E00E942D2A7DCF3D
:1090100080E00E94112A9091C606890F60E040E02E
:109020000E947E1D22CF81E00E942D2AD1CE629F18
:10903000D001739FF001829FE00DF11D649FE00D50
:10904000F11D929FF00D839FF00D749FF00D659FB1
:10905000F00D9927729FB00DE11DF91F639FB00DB0
:10906000E11DF91FBD01CF0111240895991B79E07D
:1090700004C0991F961708F0961B881F7A95C9F7A8
:1090800080950895AA1BBB1B51E107C0AA1FBB1FF7
:10909000A617B70710F0A61BB70B881F991F5A9584
:1090A000A9F780959095BC01CD01089597FB092EF5
:1090B00007260AD077FD04D0E5DF06D000201AF499
:1090C000709561957F4F0895F6F7909581959F4F24
:1090D0000895A1E21A2EAA1BBB1BFD010DC0AA1FF9
:1090E000BB1FEE1FFF1FA217B307E407F50720F011
:1090F000A21BB30BE40BF50B661F771F881F991F8C
:109100001A9469F760957095809590959B01AC01D4
:0A911000BD01CF010895F894FFCFD0
:10911A0001FFFFFFFFFFFFFFFFD012130000010056
:10912A00010001000100010001000100010001002D
:10913A0001000100010001C000800040007F20649E
:10914A0030480F04050607111210130E040506070E
:10915A00111210130409050A06070B110C120D103F
:10916A001325212326272422201D1E1B191F1C1A02
:10917A001012180F110C130E0B140D0A15160917DD
:10918A000405080306010700020320191A180C0B2C
:10919A000A090420191A180C0B0A0922212523206E
:1091AA00191A18241B1C0F0E0D04030A0C0B0908AC
:1091BA00010200201B191C1A180F0C0E0B0D0A09AC
:1091CA0026271D1E1F101211131415161705060740
:1091DA006E306E783078000100070E091C1B1215DC
:1091EA00383F363124232A2D70777E796C6B62657D
:1091FA00484F464154535A5DE0E7EEE9FCFBF2F56D
:10920A00D8DFD6D1C4C3CACD90979E998C8B82855C
:10921A00A8AFA6A1B4B3BABDC7C0C9CEDBDCD5D24C
:10922A00FFF8F1F6E3E4EDEAB7B0B9BEABACA5A23C
:10923A008F88818693949D9A2720292E3B3C35322C
:10924A001F18111603040D0A5750595E4B4C45421C
:10925A006F68616673747D7A898E878095929B9C0C
:10926A00B1B6BFB8ADAAA3A4F9FEF7F0E5E2EBECFC
:10927A00C1C6CFC8DDDAD3D4696E676075727B7CEC
:10928A0051565F584D4A4344191E171005020B0CDC
:10929A0021262F283D3A33344E49404752555C5BCC
:1092AA007671787F6A6D64633E39303722252C2BBC
:1092BA000601080F1A1D1413AEA9A0A7B2B5BCBBAC
:1092CA009691989F8A8D8483DED9D0D7C2C5CCCB9C
:1092DA00E6E1E8EFFAFDF4F30409050A06070B11C3
:1092EA000C120D1013000100010001000100010021
:1092FA00010001000100010001000100010001C09C
:10930A000080004000060601011718191A1B1C1DCF
:10931A001E1F202122233F3F3F0B0C0D0E0F101161
:10932A001213141516173F3F3F23242526272829F1
:10933A002A2B2C2D2E2F3F3F3F1718191A1B1C1DA5
:0C934A001E1F202122233F3F3F15000082
:00000001FF
